:100000000C941E060C94D2280C94FF280C944606DF
:100010000C9446060C9446060C9446060C94460630
:100020000C9446060C9446060C941B130C9446063E
:100030000C9446060C9446060C9446060C94460610
:100040000C942C290C9446060C941A2D0C945D2DBE
:100050000C9446060C9446060C9446060C944606F0
:100060000C9446060C9446062319851964196719E1
:100070006A196D1970197319761985197F19B71ACC
:10008000B91AB91AB71AB91AB91AB91AB91AB91ADA
:10009000B91AB91AB91AB91AB91AB91AB91AB91AC8
:1000A0003D1AB91AB91AB91AB91AB91AAE19B91A40
:1000B000B91AB91AB91AB91AB91AB91AB91AB91AA8
:1000C000B91AB91AB91AB91AB91AB91A491A491A78
:1000D000491A491A491A491A491A491A491AB91A98
:1000E000B91AB91AB91AB91AB91AAE19481A481A66
:1000F000481A481AB91A561A5C1A621A681A6E1AFD
:10010000741A7A1A801A8A1A941A9E1AA81AEF195F
:10011000B119B91AB91AB91AB91A3D1AB91AB91ACC
:10012000B91AB91AB91AB91AB91AB91A471A471A1B
:10013000471A471AB91A561A5C1A621A681A6E1ABE
:10014000741A7A1A801A8A1A941A9E1AA81AEF191F
:10015000B119B91AB91AB91AB91A3D1AEC1AEC1A26
:10016000EC1AEC1AEC1AEC1AEC1AEC1AEC1AEC1A5F
:10017000EC1AEC1AEC1A021C021C021C021C021CD7
:10018000021C311B3B1B451B4F1BAC1BB61BC51B6D
:10019000D61B5E1D731D7F1D881D971DBC1DC51DB3
:1001A0000E1ED71D232129212F213621442166210E
:1001B0008421456E746572206D656E752E2E2E003D
:1001C000546F67676C6564206D6963726F50504D42
:1001D00000546F67676C656420696E76657274653C
:1001E000642050504D2100546F67676C6564205443
:1001F00058206D7574696E672100546F67676C6570
:10020000642074656C656D65747279210050726F3D
:10021000746F636F6C206572726F72207769746897
:100220002052580054696D656F7574207768656E4B
:1002300020636F6E6E656374696E6720746F205201
:100240005800507265737320616E79206B65792058
:10025000746F2063616E63656C00436F6E6E6563DF
:1002600074696E6720746F2052582C20706F776508
:100270007220757020746865205258202877697440
:10028000682062696E6420706C7567206966206EF4
:100290006F74207573696E6720616C776179732064
:1002A00062696E642900546F67676C656420276912
:1002B0006D6D656469617465206F75747075742700
:1002C00000546F67676C65642027736C61766520E6
:1002D0006D6F64652700546F67676C6564202761E4
:1002E0006C776179732062696E642700546F676769
:1002F0006C65642050504D206368616E6E656C20A3
:100300006C696D69740053657420525353492069B8
:100310006E6A656374696F6E206368616E6E656C8A
:100320002028303D3D64697361626C652900536526
:10033000742050504D206D696E696D756D20737914
:100340006E630053657420626561636F6E20696E31
:1003500074657276616C0053657420626561636FC9
:100360006E2064656C617900536574206265616319
:100370006F6E206672657175656E637920696E2097
:10038000487A3A20303D64697361626C652C205074
:10039000783D504D52206368616E6E656C20782CFC
:1003A0002046783D465253206368616E6E656C202E
:1003B00078005365742050574D2073746F7020641B
:1003C000656C61792028302064697361626C6564B2
:1003D0002C20312D323535203D3D20302E317320FB
:1003E0002D2035306D696E29005365742050504DB5
:1003F0002073746F702064656C61792028302064EC
:10040000697361626C65642C20312D323535203D75
:100410003D20302E3173202D2035306D696E29003E
:10042000536574206661696C736166652064656CF0
:1004300061792028302064697361626C65642C20C6
:10044000312D323535203D3D20302E3173202D2089
:1004500035306D696E29002A2A2A2A2A2A2A2A2A50
:100460002A2A2A2A2A2A2A2A2A2A2A2A2A2A2A2AEC
:100470002A2A2A2A0052582041636B6564202D20C5
:1004800072657665727420737563636573736675E0
:100490006C21002A2A2A2A2A2A2A2A2A2A2A2A2AAD
:1004A0002A2A2A2A2A2A2A2A2A2A2A2A2A2A2A2AAC
:1004B000002A2A2A2A2A2A2A2A2A2A2A2A2A2A2AC6
:1004C0002A2A2A2A2A2A2A2A2A2A2A2A2A2A00528E
:1004D000582041636B6564202D20757064617465DC
:1004E000207375636365737366756C21002A2A2A0D
:1004F0002A2A2A2A2A2A2A2A2A2A2A2A2A2A2A2A5C
:100500002A2A2A2A2A2A2A2A2A2A0056616C696457
:100510002063686F69636573206172653A205B319F
:100520005D2D5B31365D20286368616E6E656C20E1
:10053000312D31362900536574206F7574707574D0
:1005400020666F7220706F727420005B585D2061AE
:10055000626F7274206368616E67657320616E6498
:10056000206578697420525820636F6E6669670051
:100570005B535D20736176652073657474696E6783
:100580007320746F205258005B525D20726576654F
:1005900072742052582073657474696E6773207486
:1005A0006F2064656661756C747300557365206EA9
:1005B000756D62657273205B312D445D20746F2010
:1005C0006564697420706F727473205B452D515D92
:1005D00020666F722073657474696E677300202DD6
:1005E00020726563656976657220636F6E66696700
:1005F000757261746F722C20727820737720000AF4
:100600000A6F70656E4C52536E67200053657420FC
:1006100073657269616C2062617564726174653AB8
:10062000200056616C69642063686F696365733A82
:100630002031202D20342B34202F2032202D203823
:10064000202F2033202D20382B34202F2034202D14
:10065000203132202F2035202D2031322B34202FF5
:100660002036202D20313600536574204368616E9A
:100670006E656C20636F6E6669673A20005365741F
:100680002044617461726174652028302D32293AEA
:10069000200053657420486F70206368616E6E653A
:1006A0006C7320286D61782032342C207365706162
:1006B000726174656420627920636F6D6D61732966
:1006C0002076616C69642076616C75657320312DCC
:1006D0003235353A2000536574206368616E6E656B
:1006E0006C2073706163696E6720287831306B48C5
:1006F0007A293A200053657420524620706F77653E
:10070000722028302D37293A200053657420524634
:10071000206D6167696320286865782920652E67E8
:100720002E20307844454144463030443A2000532E
:1007300065742062617365206672657175656E63AC
:10074000792028696E20487A293A20005B5A5D207A
:10075000656E746572207265636569766572206383
:100760006F6E66696775726174696F6E2075746902
:100770006C79005B465D20646973706C61792061FF
:10078000637475616C206672657175656E63696509
:10079000732075736564005B525D2063616C6375E3
:1007A0006C6174652072616E646F6D206B65792079
:1007B000616E6420686F70206C697374005B495DC2
:1007C000207265696E697469616C697A6520736508
:1007D0007474696E677320746F20736B65746368DB
:1007E0002064656661756C7473005B585D2072658A
:1007F00076657274206368616E67657320616E64EC
:100800002065786974206D656E75005B535D20739B
:100810006176652073657474696E677320746F20E8
:10082000454550524F4D20616E64206578697420B3
:100830006D656E7500557365206E756D62657273BA
:10084000205B302D395D20746F20656469742070E1
:100850006172616D657465727300202D2053797328
:1008600074656D20636F6E66696775726174696F18
:100870006E000A0A6F70656E4C52536E672000510D
:1008800029204F7574707574206265666F726520DB
:100890006C696E6B20283D465329203A2000502970
:1008A00020536C617665206D6F64652028657870D3
:1008B0006572696D656E74616C293A20004F29205C
:1008C00054696D65642042494E44206174207374FC
:1008D000617274757020203A20004E292050504DCE
:1008E000206F7574707574206C696D69746564200F
:1008F000202020203A200044495341424C454400E6
:100900004D292050504D205253534920746F20637D
:1009100068616E6E656C202020203A20004C2920F2
:1009200050504D206D696E696D756D2073796E63E1
:10093000202875732920203A200044495341424C15
:100940004544004B29204661696C736166652062ED
:100950006561636F6E20696E74762E2028312D32AA
:10096000353573293A20004A29204661696C736144
:10097000666520626561636F6E2064656C617920D5
:1009800028302D323535203D3E20313073202D204A
:100990003135306D696E293A200049292046616958
:1009A0006C7361666520626561636F6E206672714B
:1009B0002E203A200048292050574D2073746F7024
:1009C0002064656C6179202020202020203A2000BE
:1009D00047292050504D2073746F702064656C61FE
:1009E00079202020202020203A200046292046611E
:1009F000696C736166652064656C617920202020D4
:100A00002020203A200050574D206368616E6E65AB
:100A10006C200066756E6374696F6E3A2000292041
:100A2000706F72742000506F776572546F776572C3
:100A300000445446205548462033322D62697420C4
:100A400031306368004F70656E4C52536E67525878
:100A5000206D696E6920342F36636800466C7974A6
:100A6000726F6E2F4F72616E6765525820554846FF
:100A70002038636800525820747970653A20004429
:100A8000697361626C656400487A00203D3D200016
:100A900043616C63756C61746564207061636B6540
:100AA0007420696E74657276616C3A200042292068
:100AB0004D6963726F202868616C66292050504D23
:100AC000202020203A00412920496E766572746505
:100AD000642050504D20696E20202020203A0030A4
:100AE00029204D7574652062757A7A657220286DAB
:100AF0006F73746C79293A003929205365726961E2
:100B00006C2062617564726174653A00736D617224
:100B100074506F7274004672536B79005472616E38
:100B200073706172656E740044697361626C6564B0
:100B30000038292054656C656D657472793A2020FF
:100B40002020202020003729204368616E6E656CCC
:100B500020636F6E6669673A202000362920446161
:100B60007461726174652028302D32293A2020206A
:100B700000352920486F70206368616E6E656C7364
:100B80003A2020202020003429204368616E6E65C1
:100B90006C2073706163696E673A202000332920EE
:100BA000524620706F7765722028302D37293A2001
:100BB0002020003229205246206D616769633A2067
:100BC0002020202020202020003129204261736530
:100BD000206672657175656E63793A202020000089
:100BE00000000700020100000304060000000000EE
:100BF00000000001020408102040800102040810D7
:100C00002001020408102004040404040404040263
:100C10000202020202030303030303000000002395
:100C2000002600290000000000250028002B0000FD
:100C3000000000240027002A00004B2E11241FBEB4
:100C4000CFEFD8E0DEBFCDBF13E0A0E0B1E0E4EA33
:100C5000F2E602C005900D92A83CB107D9F716E064
:100C6000A8ECB3E001C01D92A239B107E1F71CE086
:100C7000CCE3DCE004C02297FE010E94542FCA336B
:100C8000D107C9F70E94872E0C9450310C940000B4
:100C900080917705813019F482E080937705809107
:100CA0007705833019F484E0809377050895A8953B
:100CB0000895DC01ED91FC910190F081E02D099502
:100CC00008952091780530917905382748E0C901C9
:100CD000880F991F37FF06C09C0151E2252750E17C
:100CE000352701C09C01415091F73093790520933D
:100CF0007805089588E380937A0580E092ECA1E07E
:100D0000B0E080937B0590937C05A0937D05B09324
:100D10007E0587E08093870580E091EAACEBB3E342
:100D200080937F0590938005A0938105B093820501
:100D300085E0809388058DEE9EEFADEABEED809351
:100D4000830590938405A0938505B0938605E9E813
:100D5000F5E080E090E0863028F4DC01AE54BC4F32
:100D60002C9101C020E0219301968831910599F7DB
:100D700082E08093A1058AE08093A205089580E037
:100D80009EECADEEB4E38093BF059093C005A093B5
:100D9000C105B093C20580E090E0A0E0B0E580938B
:100DA000C3059093C405A093C505B093C605E7ECB1
:100DB000F5E080E081938F5F8031E1F70895A0E056
:100DC000B0E0E5EEF6E00C941D2FD82F0E948229AA
:100DD0006115710581059105C9F30E94C02F10921C
:100DE0008305109284051092850510928605C4E053
:100DF000812C912C54018A94C0908305D090840555
:100E0000E0908505F0908605FE2CED2CDC2CCC24A2
:100E10000E94BB2FA50194010E94FC2E6C0D7D1D2C
:100E20008E1D9F1D609383057093840580938505B7
:100E300090938605C15001F7DD2309F450C009E8FD
:100E400015E0E801A12CB12C62E3C62ED12CE12CD7
:100E5000F12C8881882309F442C0B39419F40E94CC
:100E60007A063DC00E94BB2FA70196010E94FC2E6E
:100E7000E1E0E60FA9E8B5E08A2F801B8A1520F48F
:100E80008D918E13F9CFE9CF2091880530E0A0E154
:100E9000B7E20E94942E9B01AC01AE2FB0E00E94FD
:100EA000A32E40907F055090800560908105709042
:100EB0008205640D751D861D971D4090BF055090DD
:100EC000C0056090C1057090C205461657066806B9
:100ED000790618F2E993A39488E1A812BACFCDB7A6
:100EE000DEB7E0E10C94392F8436910520F4BC0183
:100EF00080E090E017C09C018E3B910528F42A55B4
:100F00003109AAE0B0E00CC0823D910528F4245BD1
:100F10003109A4E6B0E004C02D5C3109A8E5B2E0D7
:100F20000E94942EA4E6B0E09B01AC010E94A32E87
:100F3000089590E08C599F4F0E947407089582E0B5
:100F40008093B00085E08093B10061E083E00E946F
:100F50002F2A60E083E00E94682A08950097C9F074
:100F60009C0140E050E068E478EE81E090E00E946F
:100F7000FC2E2F3F31054105510529F020F02FEFC0
:100F800030E040E050E02093B3008091B0008061F9
:100F900003C08091B0008F7E8093B000089560E020
:100FA0008CE00E942F2A61E08BE00E942F2A61E0F2
:100FB0008DE00E942F2A60E082E00E942F2A61E0EB
:100FC00084E00E942F2A089542E050E068E476E031
:100FD00080E00E94B2280895E3E0F0E089E0809389
:100FE0005700E491E67081E0E63009F080E0089572
:100FF000CF93DF93C82F0E94EC07882381F0DFB7DF
:1010000081E080937605F8940E94570688E18093EA
:101010006000C0936000C1110E945706DFBFDF91DE
:10102000CF9108958F929F92AF92BF92CF92DF920D
:10103000EF92FF92CF93FC01C0A5EC2FE770F0E098
:10104000E658FC4FA081B0E0C7FF03C024E130E0C8
:1010500002C02FE030E0FC0197A183E1989FF001EE
:101060001124E25CFE4F80809180A280B380A20FA9
:10107000B31F20E43FE14DE750E00E94AE2EA501F2
:1010800094010E94DA2E8C2F887149F469017A014B
:10109000E0EDCE0EE7E0DE1EE11CF11C1BC0C7FF39
:1010A00005C060E47AE88CE29EE004C060E07EEE79
:1010B0008AEB9BE069017A01F8EBCF0EFBE0DF1EC3
:1010C000E11CF11CA50194010E94DA2EC20ED31E70
:1010D000E41EF51EC701B60169517C4F8F4F9F4F2B
:1010E00028EE33E040E050E00E94DA2EA8EEB3E0B4
:1010F0000E94A32ECF91FF90EF90DF90CF90BF90F2
:10110000AF909F908F9008958F3F910551F048F0D8
:10111000811522E0920738F08115934030F482E087
:10112000089580E0089581E0089583E00895A0E0A7
:10113000B0E0EDE9F8E00C94262FEB018A01B82F1E
:10114000B695A0E028813981F80120832A813B816E
:1011500021832C813D8122832E813F8123836881DD
:1011600079814A815B812C813D81EE81FF819F2FB6
:101170009295990F990F907C272F2370922B252FF2
:101180002370220F220F922B232F23702295207F72
:10119000922BF80194830B5F1F4F2896AF5FBA170D
:1011A00088F680FF24C0888199810E948408D82E07
:1011B0008A819B810E948408E82E8C819D810E94F7
:1011C0008408F82E8E819F810E948408F0E4DF9EBF
:1011D000A001112490E1E99E90011124242B282BD9
:1011E000E4E0FE9EB0011124262BF8012083CDB748
:1011F000DEB7E7E00C94422F803223E0920708F13B
:10120000883E23E0920740F48F519340E4E09695A6
:101210008795EA95E1F70895803D27E0920718F455
:101220008C5D93400895883928E0920768F4885CC3
:10123000974074E0969587957A95E1F78D509C4F8D
:10124000089580E090E008958FEF93E008958C304A
:10125000910540F4A4E0880F991FAA95E1F7885DF5
:101260009C4F0895843F23E0920718F484529C4FCA
:101270000895811524E0920740F48657934FF4E0D7
:10128000880F991FFA95E1F7089580E998E008958D
:101290009C013695279525753575821B930B9C010E
:1012A0002373337396958795969587958373937378
:1012B000820F931F9C0154E0369527955A95E1F7CC
:1012C000280F391F2F703F7041E051E0249FC0016B
:1012D000259F900D349F900D1124892F08952D98EE
:1012E000882319F000002B9A02C000002B98000000
:1012F0002D9A000008952D9A000083B12D980000CA
:10130000829581700895CF93DF93D82F5C9A2D98A2
:101310005C98C8E08D2F80780E946F09DD0FC15066
:10132000C9F72D98DF91CF9108958F770E94830997
:101330000895CF93DF93D82FC8E08D2F80780E9437
:101340006F09DD0FC150C9F72D98DF91CF91089536
:10135000CF93DF932D98C8E080E0D82FDD0F0E9457
:101360007B098D0FC150C9F7DF91CF9108950E947D
:1013700095090E94A8095C9A0895A1E0B0E0E3EC09
:10138000F9E00C942B2F806869830E94830969819E
:10139000862F0E9499095C9A2196E2E00C94472FCF
:1013A000CF93C0918305C827E82FF0E0E658FA4FA5
:1013B000678589E70E94BD096C2F8DE30E94BD09F6
:1013C0006C2F82E40E94BD09CF91089586E20E94AD
:1013D000B7090895CF93DF93EC016C818CE10E94F3
:1013E000BD096D818DE10E94BD096E818EE10E9473
:1013F000BD096F8180E20E94BD09688581E20E947B
:10140000BD09698582E20E94BD096A8583E20E9466
:10141000BD096B8584E20E94BD096C8585E20E944E
:10142000BD096D858AE20E94BD096E858EE60E9427
:10143000BD096F858FE60E94BD09688980E70E941B
:10144000BD09698981E70E94BD096A8982E70E9416
:10145000BD09DF91CF910895CF92DF92EF92FF9275
:10146000CF93DF936B017C01C11488E3D8068CE92C
:10147000E8068CE1F80628F5C701B60120E836E950
:1014800048E950E00E94DA2EE901689760E879E6C1
:1014900087E69FEF0E94B62E6C0D7D1D8E1D9F1D51
:1014A000F2E0660F771F881F991FFA95D1F721E7A1
:1014B00032E040E050E00E94DA2EF22EE32E80E48B
:1014C00021C0C701B60120E03DE241E351E00E94A6
:1014D000DA2EE901689760E073ED8EEC9EEF0E94D2
:1014E000B62E6C0D7D1D8E1D9F1D660F771F881FEC
:1014F000991F21E732E040E050E00E94DA2EF22E00
:10150000E32E80E66C2F6F71680F85E70E94BD099E
:101510006E2D86E70E94BD096F2D87E70E94BD09E9
:10152000DF91CF91FF90EF90DF90CF900895682FDB
:101530008DE60E94BD0908958F929F92AF92BF924F
:10154000CF92DF92EF92FF92CF93DF93D82F61E09B
:1015500089E00E94682A62E370E080E090E00E94E7
:10156000A52960E089E00E94682A62E370E080E0DB
:1015700090E00E94A52983E00E94B7098093750539
:1015800084E00E94B7098093740560E086E00E94C1
:10159000BD0961E087E00E94BD096FE789E00E9414
:1015A000BD0965E08AE00E94BD0965E18BE00E940B
:1015B000BD0962E18CE00E94BD096DEF8DE00E94E3
:1015C000BD0960E08EE00E94BD09DD2319F08BE2C9
:1015D00091E008C02091A10533E1239FC0011124AF
:1015E000825C9E4F0E94EA096CE880E30E94BD097C
:1015F0006FE082E30E94BD0962E483E30E94BD09BB
:101600008091A20587FF02C064E101C06AE084E323
:101610000E94BD096AE285E30E94BD096DE286E38E
:101620000E94BD0964ED87E30E94BD0960E088E384
:101630000E94BD0960E089E30E94BD09D11109C083
:10164000C0908305D0908405E0908505F0908605D4
:1016500007C0C5E9CC2EC1ECDC2EED2CCEEDFC2E66
:10166000CAE38F2C9924AA24BB24682D8C2F0E94B6
:10167000BD09682D85E08C0F0E94BD09FE2CED2C64
:10168000DC2CCC24CF5FCE3361F76FEF83E40E9474
:10169000BD096FEF84E40E94BD096FEF85E40E94ED
:1016A000BD096FEF86E40E94BD09DD2311F066E0FD
:1016B00002C0609187058DE60E94BD0960E089E760
:1016C0000E94BD09609188058AE70E94BD0960E01B
:1016D00083E70E94BD0960E084E70E94BD09D11143
:1016E00009C060917F05709180058091810590917E
:1016F000820504C060E071EA8CEB93E30E942C0A3F
:10170000DF91CF91FF90EF90DF90CF90BF90AF909F
:101710009F908F90089561E087E00E94BD0964E288
:101720008EE70E94BD0963E088E00E94BD0960E089
:1017300088E00E94BD0965E087E00E94BD0962E083
:1017400085E00E94BD0983E00E94B709809375057A
:1017500084E00E94B70980937405089583E00E9495
:10176000B7098093750584E00E94B70980937405DA
:1017700061E087E00E94BD096AE070E080E090E0EF
:101780000E94A5290E948B0B00000895CF92DF9242
:10179000FF920F931F93CF93DF931F92CDB7DEB7C6
:1017A000082F162F8EE399830E94BD09F02EC02EBC
:1017B0009981D92E8C2D8F19811738F4F6016191FA
:1017C0006F018FE70E94BD09F5CF64E085E00E94BC
:1017D000BD0983E00E94B7098093750584E00E94EB
:1017E000B709809374050E948229609370057093F5
:1017F0007105809372059093730569E087E00E94FC
:10180000BD0981E0809377050F90DF91CF911F9103
:101810000F91FF90DF90CF9008950F931F930E9438
:10182000C60B80917705813099F40E94822900913E
:101830007005109171052091720530917305601B40
:10184000710B820B930B603A76488140910548F307
:1018500080917705813031F46EE971E086EE95E094
:101860000E946E2B1F910F9108950F931F938091EB
:101870007705823021F41092770581E020C08091B5
:1018800077058130D9F40E9482290091700510916A
:1018900071052091720530917305601B710B820BED
:1018A000930B613A76488140910540F061E087E012
:1018B0000E94BD091092770582E001C080E01F916F
:1018C0000F910895CF93DF93EC014AE050E06D2F24
:1018D00070E086EE95E00E943C2C6EE286EE95E08C
:1018E0000E94402BBE0184E0769567958A95E1F7CA
:1018F0006F7077274AE050E086EE95E00E943C2C1E
:101900006EE286EE95E00E94402BBE016F70772755
:101910004AE050E086EE95E00E943C2CDF91CF91AA
:101920000895D82FC0E0CD1780F45E9A64E670E089
:1019300080E090E00E94A5295E9864E670E080E077
:1019400090E00E94A529CF5FEECF6CE271E080E0CD
:1019500090E00E94A529E6CF0F931F93CF93DF93CA
:10196000EC01062F15E0115051F0CE010E943731E5
:10197000081741F0602FCE010E943F31F4CF82E082
:101980000E94910CDF91CF911F910F910895A0E0DB
:10199000B0E0EDECFCE00C941D2F482E562EC0E07C
:1019A000D0E0612C712CE12CF12C00E010E0411012
:1019B0000CC06090D80586E4689E3001112459E17E
:1019C000E52EF12C0EEB15E01EC091E049120FC080
:1019D0006090D805E6E46E9E30011124FBE16F0EA5
:1019E000711C49E2E42EF12C0AE715E00CC082E0FC
:1019F000481209C028E1622E77247394EE24E39400
:101A0000F12C07ED15E043018C0E9D1E1092790517
:101A1000109278053401A62CA818B12CC3010196A8
:101A20006C01AE14BF04A8F4A00EB11E511006C084
:101A3000C3010E943731F501808305C0F501608143
:101A4000C3010E94AC0CF50180810E946106360141
:101A5000E2CFC301511018C0C3010E943731B82E24
:101A6000C6010E9437312B2D30E0322F2227282B40
:101A700080917805909179058217930779F4C0E0F9
:101A8000D0E05524539493CF3601609179050E949C
:101A9000AC0C60917805C6010E94AC0CC05EDE4FB4
:101AA000C13E92E0D90708F482CF852DCDB7DEB7CD
:101AB000E0E10C94392F61E082E00E94C70C0895A8
:101AC00060E082E00E94C70C8091D705853020F04D
:101AD0001092D7050E945B0D8091D7058093D805A1
:101AE000089561E080E00E94C70C61E081E00E94FF
:101AF000C70C089560E080E00E94C70C882351F075
:101B000060E081E00E94C70C882321F080917A0573
:101B1000883349F00E94BF060E947A0681E00E9445
:101B2000DF060E94710D0895882319F06AEA71E0BA
:101B300002C06EEA71E086EE95E00E946E2B089579
:101B4000FF920F931F93CF93DF9369EC7BE086EEB8
:101B500095E00E941A2B40917F055091800560917D
:101B60008105709182052AE030E086EE95E00E94C2
:101B7000432C63EB7BE086EE95E00E941A2B4091AC
:101B8000830550918405609185057091860520E15B
:101B900030E086EE95E00E94432C6DE97BE086EE16
:101BA00095E00E941A2B4AE050E06091870586EE8E
:101BB00095E00E946B2C67E87BE086EE95E00E9442
:101BC0001A2B4AE050E06091880586EE95E00E946D
:101BD0006B2C61E77BE086EE95E00E941A2BC9E84A
:101BE000D5E0F12C8E0188818823A9F0FF2031F007
:101BF00061EB71E086EE95E00E943D2B21964AE074
:101C000050E0F801608186EE95E00E94342CF39458
:101C1000F8E1FF12E7CF86EE95E00E94482B6BE5D6
:101C20007BE086EE95E00E941A2B4AE050E060913E
:101C3000A10586EE95E00E946B2C66E47BE086EEC3
:101C400095E00E941A2BE091A205E770F0E0EE0FFC
:101C5000FF1FEE57FC4F6081718186EE95E00E9478
:101C60006E2B61E37BE086EE95E00E941A2B80915B
:101C7000A2058871883069F028F4811113C068E2E8
:101C80007BE00CC0803141F0883161F46CE07BE096
:101C900005C06CE17BE002C066E17BE086EE95E08A
:101CA0000E945C2B68EF7AE086EE95E00E941A2B8A
:101CB00040917B0550917C0560917D0570917E057A
:101CC0002AE030E086EE95E00E94432C6FED7AE04A
:101CD00086EE95E00E941A2B8091C30580710E94C8
:101CE000940D66EC7AE086EE95E00E941A2B8091C6
:101CF000C30580740E94940D6DEA7AE086EE95E04B
:101D00000E941A2B8091C30580720E94940D60E995
:101D10007AE086EE95E00E941A2B8AE795E00E9411
:101D20001208AB01BC012AE030E086EE95E00E948B
:101D3000252C6BE87AE086EE95E00E941A2B8AE764
:101D400095E00E9412089B01AC0160E472E48FE010
:101D500090E00E94DA2EBA01A9012AE030E086EE76
:101D600095E00E94252C68E87AE086EE95E00E94D6
:101D70005C2BCDB7DEB7E5E00C94442F8F929F9299
:101D8000AF92BF92CF92DF92EF92FF92811107C084
:101D90006FE77AE086EE95E00E945C2B2FC090E022
:101DA0000E94740724E630E040E050E00E94DA2E02
:101DB000CA01B9012AE030E040E050E00E94DA2E8A
:101DC00049015A016B017C012AE030E0B501A40110
:101DD00086EE95E00E94252C6EE286EE95E00E944C
:101DE000402B2AE030E0B701A60186EE95E00E9484
:101DF000252C63E786EE95E00E94802BFF90EF9004
:101E0000DF90CF90BF90AF909F908F9008951F93D9
:101E1000CF93DF9365E77AE086EE95E00E941A2B78
:101E20008091A305813041F46CE57AE086EE95E07F
:101E30000E945C2B10E050C0823019F465E47AE017
:101E4000F5CF843019F461E37AE0F0CF853091F773
:101E500066E27AE0EBCFC12FD0E0C930D1050CF4B7
:101E600041C068E3610F86EE95E00E94402B6EE171
:101E70007AE086EE95E00E941A2BBE016F5F7F4FDD
:101E80004AE050E086EE95E00E94042C63E17AE09F
:101E900086EE95E00E941A2BCD55DA4FE981E032AB
:101EA00018F566E07AE086EE95E00E941A2B8981AB
:101EB000803130F06DE673E086EE95E00E943D2BB8
:101EC00069816F7070E06F5F7F4F4AE050E086EE8F
:101ED00095E00E940D2C1F5F80914C05181708F4A7
:101EE000BACF0FC061E3BECFEF70F0E0EE0FFF1F7F
:101EF000EE56FC4F6081718186EE95E00E946E2B5C
:101F0000EACF6BEE79E086EE95E00E941A2B809185
:101F1000BB050E94BE0E60ED79E086EE95E00E9462
:101F20001A2B8091BC050E94BE0E65EB79E086EE0F
:101F300095E00E941A2B8091BD050E94BE0E6AE9B1
:101F400079E086EE95E00E941A2B4091B3055091FE
:101F5000B4056091B5057091B6054115510561054F
:101F6000710539F12AE030E086EE95E00E94432CBD
:101F700067E679E086EE95E00E941A2B8091B7051E
:101F80000E949907AB01BC012AE030E086EE95E0A3
:101F90000E94432C63E479E086EE95E00E941A2BC0
:101FA0004AE050E06091B80586EE95E00E946B2C07
:101FB00006C06AE379E086EE95E00E945C2B6DE155
:101FC00079E086EE95E00E941A2B6091B905709138
:101FD000BA054AE050E086EE95E00E94552C60E09C
:101FE00079E086EE95E00E941A2B6091B20560348C
:101FF00050F470E06F5F7F4F4AE050E086EE95E06E
:102000000E940D2C06C067EF78E086EE95E00E94F6
:102010005C2B6AED78E086EE95E00E941A2B8091A9
:10202000B10580FF03C063EB71E002C067EB71E0B4
:1020300086EE95E00E946E2B6DEB78E086EE95E0E3
:102040000E941A2B8091B10582700E94940D6EE956
:1020500078E086EE95E00E941A2B8091B10584709D
:102060000E94940D6FE778E086EE95E00E941A2BAF
:102070008091B10588700E94940DDF91CF911F91DE
:1020800008950F931F93CF93DF93209149052F3F1E
:10209000A9F56FEF75E086EE95E00E941A2B88E8AF
:1020A00093E00E94620C6EED75E086EE95E00E9472
:1020B0001A2B80914A0590914B050E94620C6BEAA5
:1020C00075E086EE95E00E945C2B68E875E086EE90
:1020D00095E00E945C2B60E775E086EE95E00E943B
:1020E0005C2B6BE475E086EE95E00E945C2B86EE3F
:1020F00095E00E94482B0E94070F68C012160CF052
:1021000065C0332727FD309580914C0590E08217FC
:1021100093070CF45BC066E375E086EE95E00E94E1
:102120001A2B60914905772767FD70954AE050E0CA
:1021300086EE95E00E940D2C6BE075E086EE95E052
:102140000E941A2B10E008E280914D051817D0F577
:10215000C12FD0E0CC0FDD1FC25BDA4F288130E009
:1021600080914905992787FD909501972817390790
:1021700039F56BEB71E086EE95E00E943D2B4AE06D
:1021800050E0602F86EE95E00E94342C6FEB71E0FA
:1021900086EE95E00E943D2BE981EF70F0E0EE0FB6
:1021A000FF1FEE56FC4F6081718186EE95E00E9424
:1021B0003D2B63EC71E086EE95E00E943D2B0F5FB6
:1021C0001F5FC2CF86EE95E00E94482BDF91CF9132
:1021D0001F910F910895FF920F931F93CF93DF9359
:1021E000C9E8D5E0F12C8E0188818823D1F165EC16
:1021F00071E086EE95E00E943D2B4AE050E06F2DA5
:1022000086EE95E00E94342C62ED71E086EE95E05A
:102210000E943D2B2196F801208130E0A0E1B7E239
:102220000E94942E9B01AC01A0918805B0E00E9411
:10223000A32EAB01BC0180917F0590918005A091F8
:102240008105B0918205480F591F6A1F7B1F2AE044
:1022500030E086EE95E00E94432CF394F8E1FF1203
:10226000C2CFCDB7DEB7E5E00C94442F1092E30463
:1022700085E6E4EEF4E0DF011D928A95E9F7089522
:10228000CF93C82F8F3719F0883009F045C0E091FF
:10229000E304EE23D9F1E150E093E304F0E0EC51E4
:1022A000FB4F10826DE070E086EE95E00E945906CB
:1022B000C0E08091E304C81760F4EC2FF0E0EC512B
:1022C000FB4F608170E086EE95E00E945906CF5F7B
:1022D000F0CF60E270E086EE95E00E9459066DE076
:1022E00070E086EE95E00E945906C0E08091E3041C
:1022F000C81778F5EC2FF0E0EC51FB4F608170E0EF
:1023000086EE95E00E945906CF5FF0CF67E086EE3B
:1023100095E00E94402B1DC08B3119F40E943611AC
:102320001AC08D30C1F08A30B1F08091E304843658
:1023300068F76C2F70E086EE95E00E945906E091F8
:10234000E30481E08E0F8093E304F0E0EC51FB4F57
:10235000C08380E001C081E0CF910895CF93C82F62
:102360000E9482296093CC047093CD048093CE04A4
:102370009093CF04C093E104CC2329F040E051EEC8
:1023800060E070E004C040E855E260E070E086EE96
:1023900095E00E94CA2DCF9108959091D004492FC5
:1023A0004F7050E0BA016F5F7F4F292F30E0E4E0BB
:1023B00035952795EA95E1F76217730759F0FA0109
:1023C000EF52FB4F808381E0890F8F70907F892BC4
:1023D0008093D00408956EE770E086EE95E00E9449
:1023E00059060895A3E1B1E0E8EFF1E10C941E2F46
:1023F000E9E8F5E0712C8191882321F0739428E1BC
:102400007212F9CF66ED71E086EE95E00E946E2BB8
:102410004AE050E0672D86EE95E00E946B2C80E04C
:102420000E949C0A0E948B0B8E010E5F1F4FC12CD5
:10243000D12C7601C39466246A945C2C0E94762980
:102440004B015C012091880530E0A0E1B7E20E94D9
:10245000942E9B01AC01C701B6010E94B62E2091BB
:102460007F05309180054091810550918205620F72
:10247000731F841F951F2091BF053091C0054091A7
:10248000C1055091C205261737074807590718F4A8
:10249000F801608225C08C2D0E94D00961E070E0B7
:1024A00080E090E00E94A529F80110820E94762920
:1024B000681979098A099B09643F71408105910572
:1024C00040F40E94E609F8019081981778F780831C
:1024D000EDCF50FE03C05D985E9A02C05D9A5E9893
:1024E0002FEFC21AD20AE20AF20A0F5F1F4F8FEFD4
:1024F000C816D104E104F10409F09FCFCE019395F1
:10250000FC01D82E7FEF68EC2E2F281B271510F02A
:1025100051E056C0DE01129651E02FEF41E03D91AF
:10252000321710F0322F01C0452F5F5F5F3F11F06F
:10253000232FF5CF4193242F30E0A1E0B0E0AC0F82
:10254000BD1FA20FB31F5C93413079F0DE01A20FD3
:10255000B31F5C93423049F0AFEFBFEFAC0FBD1F2C
:10256000A20FB31F6C934E3F78F6A2E0B0E0AC0F21
:10257000BD1FA20FB31F7C934D3F30F6A3E0B0E028
:10258000AC0FBD1FA20FB31F6C93BECF452F242FDE
:1025900030E0FC01E20FF31F6081AFEFB0E0AC0F61
:1025A000BD1FA20FB31F2C91621748F44150DC01EC
:1025B000A40FB11D2C9120836C934111E8CF5F5F74
:1025C000571520F3372D369520E0231770F4DC01E2
:1025D000A20FB11D4C91522F530FFC01E50FF11DBD
:1025E00050815C9340832E5FF0CFF9E8EF2EF5E049
:1025F000FF2E8C01802F8D19871598F4F801C1905A
:102600008F014AE050E06C2D86EE95E00E94342C5C
:102610006CE286EE95E00E94402BF701C1927F01AB
:10262000E9CF86EE95E00E94482B81E0CD5EDE4F3B
:10263000EFE00C943A2F1F920F920FB60F921124D5
:102640001F932F933F934F935F936F937F938F933A
:102650009F93AF93BF93CF93DF93EF93FF93C0917B
:102660008600D09187008091870490918804209102
:10267000A904211155C09E01281B390B8091C30567
:102680009091C405A091C505B091C60585FD02C015
:1026900036952795253C49E03407B8F140910A0169
:1026A00050E060E070E02CE1B695A795979587958E
:1026B0002A95D1F70097A105B10521F481E090E0BA
:1026C000A0E0B0E084179507A607B707D8F480917B
:1026D0000A018F3FB9F040E080910A01481780F469
:1026E000842F90E0880F991FFC01E757FB4F208152
:1026F0003181FC01E55FFE4F318320834F5FECCFDA
:102700001092AA0410920A010BC02D3B82E03807F8
:1027100020F080910A018031D8F08FEF80930A0178
:10272000D0938804C0938704FF91EF91DF91CF91FC
:10273000BF91AF919F918F917F916F915F914F91D9
:102740003F912F911F910F900FBE0F901F901895E2
:1027500010910A0181E0810F80930A01C9010E9452
:10276000FC08E12FF0E0EE0FFF1FE757FB4F9183CE
:102770008083D6CF83E0809380008AE980938100B4
:102780008091C30586FD05C080918100806480939F
:1027900081008FEF9FEF9093890080938800809154
:1027A0006F00806280936F000895CF93DF930E9443
:1027B000600D8091D805843039F58FE00E949B2A06
:1027C000C1E0D0E0892B11F4C0E0D0E080E10E94AC
:1027D0009B2A892B19F082E090E002C080E090E013
:1027E0008C2B9D2B8230910539F08330910539F087
:1027F000019739F481E006C01092D80505C082E047
:1028000001C083E08093D805DF91CF9108956F30A8
:1028100018F086958058089589E0689F802D1124CE
:102820000895A0E0B0E0E7E1F4E10C94252FC82F73
:102830000E948229009138041091390420913A04B1
:1028400030913B046B017C01C01AD10AE20AF30A01
:102850009701860149E8C41643E1D406E104F10476
:1028600010F010923C046093380470933904809304
:102870003A0490933B042091A9048FEF820F823099
:10288000E8F5E0913C04EE2309F46EC1E13011F467
:1028900082E0D8C1E03178F581E08E0F80933C046E
:1028A000F0E0E757FB4FC083803109F0D4C1EBE87B
:1028B000F4E0213029F4A181A695A695808108C075
:1028C00080819181A92FA695A695A6959695879525
:1028D000A03148F4B0E090E0AA0FBB1FA55FBE4F47
:1028E00011969C938E931092AA04329684E0E93953
:1028F000F807F9F6B0C110923C04ADC1233009F0DD
:1029000023C1E0913C04E11118C0CF3009F011C19E
:102910000E9476290091B7041091B8042091B9045F
:102920003091BA04601B710B820B930B62307105FE
:102930008105910508F089C1FCC0E73148F481E0C8
:102940008E0F80933C04F0E0E857FB4FC083F1C04A
:10295000E73109F0ECC0C111EAC040E050E0ABE063
:10296000CA01B3E0880F991FBA95E1F7A49F9001BF
:10297000A59F300D1124F901E757FB4F6081E181DC
:102980007E2F777075956795FC01EE0FFF1FE55F51
:10299000FE4F71836083F901E657FB4FB081B69516
:1029A000B695B695E181FE2FF295FF0FF07E6F2F61
:1029B0006B2BE695E695E6957E2F77707595679576
:1029C000FC01EE0FFF1FE35FFE4F71836083F9018F
:1029D000E557FB4FB081B295B695B695B370C181FE
:1029E000DC2FDD0FDD0F6D2F6B2BC295C695C695C5
:1029F000C370E281E170EE0FEE0F7E2F7C2B759598
:102A00006795FC01EE0FFF1FE15FFE4F718360834E
:102A1000F901E357FB4FB081B695E181FE2FF795A1
:102A2000FF27F7956F2F6B2BE6957E2F77707595A7
:102A30006795FC01EE0FFF1FEF5EFE4F7183608311
:102A4000F901E257FB4FB081B295BF70E181FE2FD3
:102A5000F295F07F6F2F6B2BE295EF707E2F7770E2
:102A600075956795FC01EE0FFF1FED5EFE4F7183BC
:102A70006083F901E157FB4FB081BB1FBB27BB1F30
:102A8000C181DC2FDD0F6D2F6B2BCC1FCC27CC1F12
:102A9000E281E370EE0F7E2F7C2B75956795FC012C
:102AA000EE0FFF1FEB5EFE4F71836083F901EF565F
:102AB000FB4FB081B695B695E181FE2FF295FF0FE1
:102AC000FF0FF07C6F2F6B2BE695E6957E2F7770CE
:102AD00075956795FC01EE0FFF1FE95EFE4F718350
:102AE0006083F901EE56FB4F2081229526952770D1
:102AF0003181E32FEE0FEE0FEE0F6E2F622B732F4F
:102B000072957695777075956795FC01EE0FFF1FAE
:102B1000E75EFE4F718360834F5F5F4F4230510528
:102B200009F01ECF80919F0483FF1092AA04109297
:102B30003C040E9476296093B7047093B804809394
:102B4000B9049093BA0487C0243009F084C060911E
:102B50003C0461110BC0C83AB1F41092790510928F
:102B6000780588EA0E94610681E06CC0613019F442
:102B7000C093370404C0623031F4C09336048C2F04
:102B80000E9461065AC0E09136042E2F30E0220FD9
:102B9000331F462F50E0C9010296841795073CF079
:102BA000633268F7FA01EA57FB4FC083E8CF2D5F25
:102BB0003F4F8C2F90E06091780570917905421716
:102BC000530749F4982F88278627972790937905EC
:102BD0008093780532C06817790769F580913704CA
:102BE000813049F5E13118F080E180933604F090AE
:102BF0003604CAE8D4E000E010E00F15D0F4FE017E
:102C00003197808190E0982F88272881822B63E07C
:102C1000969587956A95E1F70E94FC08F801EE0FFA
:102C2000FF1FE55FFE4F918380830F5F1F4F22964A
:102C3000E4CF1092AA0410923C0480913C048823B3
:102C400051F08F5F80933C0406C080913C048F5FFD
:102C500080933C046ECFCDB7DEB7E8E00C94412FF3
:102C6000CF93DF93E82FF0E0E254FA4FE185E031B3
:102C700050F4F894F0E0EE0FFF1FE55FFE4F808107
:102C8000918178945DC08EE08E0F8B3058F4F0E027
:102C9000E25FF10924E62E9FC0012F9F900D1124C1
:102CA0000C964EC0E03F09F446C038F4E13181F0A3
:102CB000E23191F0E03139F409C0ED3FB1F1EE3F7E
:102CC000B9F1E13F79F180E092E03AC082E101C0E0
:102CD00083E10E94C42A34C08FE00E949B2AC1E095
:102CE000D0E0892B11F4C0E0D0E080E10E949B2A63
:102CF000892B19F082E090E002C080E090E08C2BFC
:102D00009D2B8230910541F08330910541F0019770
:102D1000A9F086EA92E014C08CE090E011C089E549
:102D200091E00EC086E090E00BC08AEF93E008C00F
:102D30008FEF93E005C080E090E002C084EF93E065
:102D4000DF91CF910895A2E2B0E0E9EAF6E10C94B8
:102D50001B2F9E012F5F3F4F80E1D9011D928A9565
:102D6000E9F764E072E086EE95E029A33AA30E94B9
:102D70006E2B0E94AE0B1D8A1E8A1F8A188E312C64
:102D8000212C00E0812C912C5401412C74E7572E0A
:102D90007BE8672E72E3772EE0E5CE2EE3ECDE2EA5
:102DA000E12CF12C84EF91E0A0E0B0E08D8F9E8FBC
:102DB000AF8FB8A380E09EECADEEB4E3898F9A8F1D
:102DC000AB8FBC8F80E094E7ABE8B2E3898B9A8B42
:102DD000AB8BBC8B86EE95E00E94822C892B09F48C
:102DE000E1C086EE95E00E94AF2C9C0133272C3287
:102DF000310509F442C0ACF42332310509F0ABC00F
:102E000019821A821B821C821D821E821F821886D2
:102E100019861A861B861C861D861E861F86188AA2
:102E200060C02434310529F02335310509F4B2C0DE
:102E300092C064E486EE95E00E94402B2AE030E0E8
:102E400040E054E76BE872E386EE95E00E94CE2BFB
:102E50006CE286EE95E00E94402B2AE030E040E0F4
:102E60005EEC6DEE74E386EE95E00E94CE2B6CE294
:102E700086EE95E00E94802BADCF0F5F043009F005
:102E8000A9CF29813A814B815C81A8EEB3E00E94F1
:102E9000A32E698B7A8B8B8B9C8B2D813E814F81EE
:102EA00058850E94A32E698F7A8F8B8F9C8F2985DE
:102EB0003A854B855C852D8F3E8F4F8F58A32D858E
:102EC0003E854F8558890E94A32E6B017C0160329C
:102ED0003EE473078105910530F462E38CE10E94C2
:102EE000BD0900E077CF603345E7740781059105A0
:102EF00010F462E2F3CF60345CE975078105910557
:102F000010F466E2EBCF80E5C81683ECD806E10446
:102F1000F10410F462E1E2CF90E6C9169AEED90608
:102F2000E104F10410F465E1D9CFA0E7CA16A1E1EC
:102F3000DA06A1E0EA06F10410F461E0CFCFB0EACE
:102F4000CB16B6E8DB06B1E0EB06F10410F463E063
:102F5000C5CF65E0C3CF10ED180F1A3008F03ACF97
:102F6000E1E0F0E0EC0FFD1F24E0029FE00DF11D19
:102F700011242081318142815381AAE0B0E00E9476
:102F8000A32E610F711D811D911D6083718382834A
:102F9000938320CF49885A886B887C88812C912C18
:102FA000540118CF81149104A104B10489F4C30120
:102FB000B2010E942C0A61E070E080E090E00E9483
:102FC000A5291D8A1E8A1F8A188E312C22242A9434
:102FD0008D8D9E8DAF8DB8A188169906AA06BB0669
:102FE000D0F40E94E6092D893E894F89588D280F1B
:102FF000311D411D511D2D8B3E8B4F8B588F381627
:1030000008F4382E821508F4282E3FEF831A930A0D
:10301000A30AB30A56C0C301B20128EE33E040E070
:1030200050E00E94DA2EBA01A9012AE030E086EED3
:1030300095E00E94252C6CE286EE95E00E94402BE4
:103040004AE050E0632D86EE95E00E94342C6CE25D
:1030500086EE95E00E94402B6D897E898F89988D40
:10306000A50194010E94DA2EBA01A9012AE030E0FC
:1030700086EE95E00E94252C6CE286EE95E00E949B
:10308000402B4AE050E0622D86EE95E00E94342C01
:103090006CE286EE95E00E94802B4C0C5D1C6E1C51
:1030A0007F1C898D9A8DAB8DBC8D84159505A605E9
:1030B000B70520F449885A886B887C88812C912C2C
:1030C000540129893A894B895C89283E334041055E
:1030D000510509F07FCEA296E2E10C94372FACE1C6
:1030E000B0E0E5E7F8E10C94252F0E9482296B01FE
:1030F0007C0181E00E949C0A14E703E0198361E0EF
:10310000CE0101960E940D0C009377050E948B0B57
:103110006AEF70E080E090E00E94A5298091770539
:10312000833089F486EE95E00E94822C892B59F435
:103130000E9482296C197D098E099F096038734CA1
:10314000894C9140D8F280917705833009F44FC0C3
:103150008FE70E9495090E94A8098983843511F0A0
:1031600083E05CC00E94A80910924A0580934B0539
:103170000E94A80920914A0530914B05280F311D66
:1031800030934B0520934A050E94A80980934C0573
:103190000E94A80980934D05813110F7F12C0F2D65
:1031A00010E080914D0590E0880F991F08171907CE
:1031B00040F40E94A809F801E25BFA4F8083F3947F
:1031C000EECF80E7898361E0CE0101960E940D0C6D
:1031D00083E0809377050E948B0B62E370E080E0D0
:1031E00090E00E94A52980917705833011F482E058
:1031F00015C08FE70E9495090E94A8098983803530
:1032000009F0AECF03EA15E00E94A809F801819306
:103210008F01F5E00E3B1F07B9F781E06C96E8E0FF
:103220000C94412F80914905992787FD9095A92FEE
:10323000B92FFC013196EB30F10508F066C0EC5C6B
:10324000FF4F0C94522F62E778E086EE95E00E94E3
:103250005C2B88E893E00E94620C6AE578E086EED9
:1032600095E00E945C2B65E378E086EE95E00E9495
:103270005C2B6BE078E086EE95E00E945C2B6AEEBA
:1032800077E086EE95E00E945C2B6DEB77E086EEB2
:1032900095E00E945C2B67E977E086EE95E00E945E
:1032A0005C2B63E777E086EE95E00E945C2B6CE494
:1032B00077E086EE95E00E945C2B86EE95E00E941A
:1032C000482B0E94A00D21C06FE277E01AC06AE08F
:1032D00077E017C065EF76E014C066ED76E011C0C8
:1032E00062E976E00EC06DE776E00BC068E676E056
:1032F00086EE95E00E945C2B62E276E002C06CE014
:1033000076E086EE95E00E945C2B6AE070E080E05B
:1033100090E00E94A52986EE95E00E94822C892BE0
:1033200029F086EE95E00E94AF2CF5CF0895ACE130
:10333000B0E0EDE9F9E10C94252F909149059F3F0C
:1033400009F023C1482F50E0FA013A97EF36F10512
:1033500008F00FC1E15CFF4F0C94522F61E172E065
:10336000A0C06DE172E086EE95E00E946E2B85E7CD
:1033700089838BE1E3EAF5E0DE01129601900D927C
:103380008A95E1F76CE1CE0101960E940D0C0E9436
:103390008B0B83E08093770568EC70E080E090E031
:1033A0000E94A52980917705843009F0E2C08FE75B
:1033B0000E9495090E94A8098983853509F0D9C022
:1033C0006DEE74E086EE95E00E945C2B6FEC74E08D
:1033D00086EE95E00E945C2B61EB74E096C065E39D
:1033E00072E086EE95E00E946E2B89E6898361E0AB
:1033F000CE0101960E940D0C0E948B0B83E08093FE
:10340000770568EC70E080E090E00E94A52980914B
:103410007705843009F0ADC08FE70E9495090E94BE
:10342000A80989838E010E5F1F4F7E014DE1E40ED6
:10343000F11C0E94A809F80181938F01EE15FF0588
:10344000C1F78BE1FE013296A3EAB5E001900D923F
:103450008A95E1F78981893409F08BC063E974E0CA
:1034600086EE95E00E945C2B65E774E086EE95E0C1
:103470000E945C2B67E574E048C06FE472E086EE62
:1034800095E00E946E2B8EEF8093490572C08052AA
:103490008750805390914C05981708F066C06EE5F0
:1034A00072E086EE95E00E946E2B63C084E180930B
:1034B000490560E274E029C085E18093490569EE21
:1034C00073E023C086E18093490562EB73E01DC081
:1034D00087E18093490568E673E017C088E180932F
:1034E000490567E573E011C089E18093490563E40C
:1034F00073E00BC08AE1809349056EE273E005C07A
:103500008BE18093490566E073E086EE95E00E94CA
:103510005C2B2FC06CEE72E086EE95E00E945C2B77
:103520008091B10591E01DC066ED72E086EE95E0F8
:103530000E945C2B8091B10592E013C061EC72E0B7
:1035400086EE95E00E945C2B8091B10594E009C065
:1035500066EA72E086EE95E00E945C2B8091B105F0
:1035600098E089278093B1058FEF809349050E94E9
:10357000411086EE95E00E94822C892B09F45AC1F5
:1035800086EE95E00E94AF2CF4CF0E944011882374
:1035900009F450C18091E304811104C08FEF80933E
:1035A000490540C140E050E060E070E084EE94E006
:1035B0000E94C92F40914905042F112707FD10953E
:1035C000212F312FF8013197EB31F10508F01AC1A5
:1035D000E255FF4F0C94522F552747FD50952091EF
:1035E0004C0530E0241735070CF40CC18B019C010D
:1035F0000150110921093109003211052105310558
:1036000058F0C0904D05EFE4F5E0F12CD12CA8E284
:10361000EA2E415051090FC0FA01ED55FA4F6150A1
:103620006083D8C0DF0111972C9130E02417350753
:1036300029F0F3943296FC10F5CFCAC00E2D10E09D
:1036400020E030E0061717072807390741F42081EA
:10365000DA01AD55BA4F11962C93DD24D394E3943F
:10366000E8CF6F3F71058105910511F008F0CAC0E0
:103670006093BB05AFC06F3F71058105910511F0E7
:1036800008F0C0C06093BC05A5C06F3F71058105FF
:10369000910511F008F0B6C06093BD059BC0209164
:1036A000E40420622037E9F440E050E060E070E09C
:1036B00085EE94E00E94C92F9B01AC01DC01CB0197
:1036C0000197A109B1090897A105B10508F0ADC09E
:1036D000A4EDB0E30E94A32E6A5E7C4A8A46954E12
:1036E00024C02636E9F440E050E060E070E085EE6A
:1036F00094E00E94C92F9B01AC01DC01CB01019732
:10370000A109B1090797A105B10508F08EC0A8EA83
:10371000B1E60E94A32E645E7C438E46944E05C0A3
:10372000611571058105910571F08B019C0114579C
:103730002B4832430130FAE51F07F2E62F07F2E08B
:103740003F0708F05FC06093B3057093B4058093A2
:10375000B5059093B6053EC06F3F71058105910593
:1037600011F008F04FC06093B70534C08B019C0185
:1037700001501109210931090F3F110521053105BA
:1037800008F040C06093B80525C08B019C01045C23
:103790001940210931090D344DE114072105310586
:1037A00028F47093BA056093B90514C061157105CA
:1037B0008105910521F48FEF8093B2050BC0613430
:1037C000710581059105F0F461506093B20502C066
:1037D000DD20C1F08091E20481111AC0809183053F
:1037E00090918405A0918505B09186050196A11D53
:1037F000B11D8093830590938405A0938505B093B4
:10380000860506C060E772E086EE95E00E946E2BAA
:103810000E9436118FEF809349056AE086EE95E0AD
:103820000E94802B0E94411005C061E070E080E0A2
:1038300090E07BCF6C96E8E00C94412F6AE572E053
:1038400086EE95E00E945C2B62E472E086EE95E0E5
:103850000E945C2B86EE95E00E94822C892B31F031
:1038600086EE95E00E94AF2C0E9497190E946F1877
:10387000823029F0833051F46DE072E002C064E2DE
:1038800072E086EE95E00E945C2B08958FEF8093A6
:1038900049051092E2040E944110809149058E3F33
:1038A00069F086EE95E00E94822C892BB1F386EEBA
:1038B00095E00E94AF2C0E949719EFCF08950F93C7
:1038C0001F93109149051F3F09F0D2C0893409F4B4
:1038D00057C000F5883309F469C058F4803309F4FF
:1038E00077C008F061C08B3109F440C08132B1F17A
:1038F000B9C0813409F487C030F4893309F466C053
:10390000803461F1AFC0823409F48EC0863409F48A
:1039100048C0A8C0823609F487C078F4883531F1F0
:1039200028F48235C1F18335E1F09CC08A3509F471
:1039300094C0813609F467C095C0823761F128F4DC
:10394000863679F18936E1F08DC0883779F08A378B
:1039500009F483C0833709F085C003C061E172E0D8
:1039600015C00E94710D6EE872E004C00E947A0DCD
:1039700068EA72E086EE95E00E946E2B8EEF70C0D2
:103980000E947A060E94BF0667EC72E086EE95E020
:103990000E946E2B67C081E00E94DF0660EE72E03D
:1039A000F5CF0E94EB105EC080535AC06AEF71E001
:1039B00086EE95E00E945C2B9091A20588E0890F2D
:1039C0008871977E892B8093A2051AC089E048C030
:1039D00067EE71E086EE95E00E945C2B8091C30556
:1039E0009091C405A091C505B091C60520E182273C
:1039F0008093C3059093C405A093C505B093C605F5
:103A0000109349052FC061ED71E086EE95E00E94AC
:103A10005C2B8091C3059091C405A091C505B09120
:103A2000C60540E4842710C060EC71E086EE95E0A6
:103A30000E945C2B8091C3059091C405A091C5059F
:103A4000B091C60520E282278093C3059093C405F8
:103A5000A093C505B093C60502C00E941E1C8FEF3F
:103A600080934905809149058E3F09F0D4C0DDC09F
:103A70000E944011882309F4D8C08091E304811189
:103A800004C08FEF80934905C6C040E050E060E07D
:103A900070E084EE94E00E94C92F0091490511273F
:103AA00007FD1095212F312FF8013197E930F105ED
:103AB00008F0B4C0E753FF4F0C94522F8B019C01C8
:103AC000015014472B4832430F3F194522463240DC
:103AD00008F0A4C060937F057093800580938105F2
:103AE0009093820577C060938305709384058093DB
:103AF00085059093860581E08093E2046BC0683071
:103B000071058105910508F089C06093870562C041
:103B10008B019C0101501109210931090A3011055D
:103B20002105310508F07AC06093880553C061EB28
:103B300071E084EE94E00E94033110E0009799F068
:103B40000E94DD30009779F0183130F4E12FF0E079
:103B5000E658FA4F87871F5F61EB71E080E090E0E5
:103B60000E940331EBCF1831A8F5E12FF0E0E658C1
:103B7000FA4F17861F5FF7CF6530710581059105F4
:103B800008F04CC06093A10525C08B019C01015039
:103B90001109210931090630110521053105F0F51A
:103BA0002091A205287F262B2093A20513C08B010C
:103BB0009C0101501109210931090115124C2140C4
:103BC000310560F560937B0570937C0580937D05DE
:103BD00090937E058091E204811113C0809183054A
:103BE00090918405A0918505B09186050196A11D4F
:103BF000B11D8093830590938405A0938505B093B0
:103C000086050E9436118FEF809349056AE086EEA3
:103C100095E00E94802B0E94121907C060E772E0B5
:103C200086EE95E00E946E2BECCF1F910F910895C8
:103C30008FEF809349051092E2040E94121980913F
:103C400049058E3F69F086EE95E00E94822C892B13
:103C5000B1F386EE95E00E94AF2C0E945F1CEFCF7F
:103C60006AE070E080E090E00E94A52986EE95E091
:103C70000E94822C892B29F086EE95E00E94AF2CC1
:103C8000F5CF0895CF93C82F682F86EE95E00E9458
:103C9000DC2C90916E059C2790936E05CF91089532
:103CA000A1E0B0E0E6E5FEE10C942B2F99830E94A1
:103CB000421E9981892F0E94421E2196E2E00C94B7
:103CC000472F1F93CF93DF93182FEB0110926E05B0
:103CD00065EB70E086EE95E00E94590662E670E0C2
:103CE00086EE95E00E945906812F0E94421ECE0169
:103CF0000E94501EDF91CF911F91089560916E0533
:103D000086EE95E00E94DC2C0895A1E2B0E0EBE89D
:103D1000FEE10C94272F7B018A018C3009F453C1FA
:103D200008F040C0863009F4BCC018F5833009F4AF
:103D300091C070F4813009F472C0823009F04AC237
:103D40006BE170E082E00E94611E03EA15E078C03A
:103D5000843009F487C0853009F03CC260914D057C
:103D600070E0660F771F85E00E94611E0EE415E08B
:103D700086C0893009F4A7C070F4873009F49BC06D
:103D8000883009F027C261E070E088E00E94611E7F
:103D90008091D80525C28A3009F4CAC08B3009F455
:103DA000F2C018C28A3609F475C1D8F4873609F40E
:103DB0003AC138F4853609F40EC1863609F41FC1BC
:103DC00009C2883609F437C1893609F003C261E0B7
:103DD00070E089E60E94611E0E947A060E94BF067A
:103DE000F7C18D3609F4D4C138F48B3609F491C18A
:103DF0008C3609F49AC1EEC18E3609F4DEC1873CD7
:103E000009F0E8C161E070E087EC0E94611E81E08A
:103E10000E94421E0E947E1E10926F05E5C169E25B
:103E200070E081E00E94611E0AE715E0F8018191CF
:103E30008F010E94421EF5E0033A1F07B9F7D2C175
:103E4000F80181918F010E94421EF5E00E3B1F0791
:103E5000B9F7C8C161E070E083E00E94611E0E9472
:103E60006F18BEC161E070E084E00E94611E81E0D5
:103E70000E94421E0E947E1E0E94A316B5C1809120
:103E80004D0590E0880F991F98012E543540281752
:103E9000390708F0A7C1F80181918F010E94421EE5
:103EA000EECF62E070E086E00E94611E88E893E059
:103EB0000E94501E97C161E070E087E00E94611E81
:103EC00080914C058DC186E6898361E0CE01019623
:103ED0000E940D0C0E948B0B83E08093770568ECA9
:103EE00070E080E090E00E94A52980917705843001
:103EF000D9F48FE70E9495090E94A8098983863426
:103F000069F460E270E089E00E94611E10E20E94A4
:103F1000A8090E94421E1150D1F764C161E070E00F
:103F200089E00E94611E54C161E070E089E055C1E2
:103F300069E170E08AE00E94611E81E08093BE0525
:103F4000209176058091C3059091C405A091C50587
:103F5000B091C605222311F0806801C08F7780934D
:103F6000C3059093C405A093C505B093C6050EEB99
:103F700015E0F80181918F010E94421EF5E0073D96
:103F80001F07B9F72FC161E270E08BE00E94611E4C
:103F90008091AA048F3F39F08091AA0491E0980F94
:103FA0009093AA0402C08091AA040E94421E10E0CD
:103FB000812F0E9430160E9427090E94501E1F5F09
:103FC0001031B1F70FC161E070E08CE00E94611E1A
:103FD0008091D70505C161E070E085E60E94611E11
:103FE00089E2E816F10409F0FAC0D801EAE7F5E041
:103FF0008D91819385E0E33AF807D1F7E9C061E05C
:1040000070E086E60E94611EEBE1EE16F10409F015
:10401000E6C0D801E3EAF5E08D91819385E0EE3BBF
:10402000F807D1F7D5C061E070E087E60E94611E15
:104030000E94710DCDC061E070E088E60E94611EB3
:1040400085E789838BE1E3EAF5E0DE0112960190D2
:104050000D928A95E1F76CE1CE0101960E940D0C5C
:104060000E948B0B83E08093770560E273E080E031
:1040700090E00E94A52980917705843009F0AFC0B7
:104080008FE70E9495090E94A8098983853509F068
:10409000A6C09EC061E070E08AE60E94611E89E6CB
:1040A000898361E0CE0101960E940D0C0E948B0B6A
:1040B00083E08093770560E273E080E090E00E9407
:1040C000A52980917705843009F089C08FE70E9487
:1040D00095090E94A80989838E010E5F1F4F7E01FA
:1040E000EDE1EE0EF11C0E94A809F80181938F0109
:1040F000EE15FF05C1F78BE1FE013296A3EAB5E0AC
:1041000001900D928A95E1F78981893409F067C0A1
:104110005FC061E070E08BE60E94611EF801808163
:104120008093D8050E947A0D53C061E070E08CE660
:104130000E94611EF0E2EF16F10461F487E68983C4
:1041400080E2F801DE01129601900D928A95E1F766
:1041500061E203C087E4898361E0CE0101960E9499
:104160000D0C0E948B0B83E0809377056CE474E068
:1041700080E090E00E94A52980917705843079F550
:104180008FE70E9495090E94A809873441F520C055
:1041900061E070E08DE60E94611E89E1E816F1049D
:1041A000F1F4D801EEEBF5E08D91819385E0E73DE8
:1041B000F807D1F70E94BA130BC061E070E08EE6F9
:1041C0000E94611EF80180818093D7050E945B0DDB
:1041D00081E006C061E070E08AEC0E94611E80E030
:1041E0000E94421E0E947E1EA196E6E00C94432F80
:1041F000A0E0B0E0EEEFF0E20C94252FCAECD3E0A3
:1042000014E606E035E0F32E44E0E42E53E0D52E2C
:1042100062E0C62E86EE95E00E94822C892B09F47E
:104220009BC086EE95E00E94AF2C282F809335042A
:104230004091340450E04730510560F7FA01EE52E6
:10424000FF4F0C94522F853B29F781E08093340473
:10425000E1CF823609F07DC0C0923404DBCF809379
:10426000330480933204D0923404D4CF9C0133279A
:104270003093310420933004909132049827909326
:104280003204E0923404C6CF382F22274091300404
:1042900050913104242B352B30933104209330047A
:1042A00090913204982790933204F092340425368A
:1042B000310508F4AFCF61E070E08CEC0E94611E24
:1042C00081E00E94421E0E947E1E43C020912E0467
:1042D00030912F04F901E653FC4F80839091320412
:1042E000982790933204C901019690932F048093EC
:1042F0002E0420913004309131048217930708F482
:1043000089CF0093340486CF8091320482130BC08E
:1043100060912E0470912F044AEC53E08091330495
:104320000E94851E0DC062E070E08BEC0E94611E51
:10433000809133040E94421E80916E050E94421EAD
:10434000FE01812F11928A95E9F710922F041092A5
:104350002E04109234045ECFCDB7DEB7E8E00C94A3
:10436000412F81E080936F0580916F05882349F08C
:1043700086EE95E00E94822C892BB1F30E94F820F2
:10438000F3CF0895AAE2B0E0E8ECF1E20C94232F19
:104390000E9476296B017C0181E00E949C0A86EED6
:1043A00095E00E94822C892B29F086EE95E00E94F0
:1043B000AF2CF5CF5E9811E072E6B72EE9E2AE2E93
:1043C00003E00E9476296C197D098E099F09693CDA
:1043D000710581059105D0F11123C1F10E94762963
:1043E0006B017C015D9A80ED97E00E94AE07B98277
:1043F000EAE7F5E0DE0112968A2D01900D928A958A
:10440000E1F76AE2CE0101960E940D0C5D9880E012
:1044100090E00E94AE07009377050E948B0B62E349
:1044200070E080E090E00E94A529809177058430BB
:1044300061F4009377058FE70E9495090E94A8090F
:1044400011E0823419F410E001C011E08EE00E9406
:104450009B2A892B81F411E00EC05E9A5D9A86EE4C
:1044600095E00E94AF2C8D309105A9F05CF40A977D
:1044700091F05E985D9886EE95E00E94822C892BE3
:1044800061F79FCF8332910579F08234910589F7E6
:104490000E94B121EECF62EB71E086EE95E00E94C2
:1044A0005C2B0E94181EE5CF0E94A316E2CF8F92CC
:1044B0009F92AF92BF92CF92DF92EF92FF921F93A3
:1044C000CF93DF938EE00E949B2A892B09F089C04D
:1044D00068EC70E080E090E00E94A52980E090E028
:1044E0000E94AE070E9476294B015C016B017C01A2
:1044F00080ECC80E82E1D81EE11CF11C0E947629D6
:104500006C157D058E059F0530F48EE00E949B2A78
:10451000892BA1F364C08EE00E949B2A892B09F0AD
:104520005EC080ED97E00E94AE070E9476296B0185
:104530007C01D0E0C1E088E4880E86E2981EA11CD0
:10454000B11C11E08EE00E949B2A892B21F58C146E
:104550009D04AE04BF0430F480ED97E00E94AE07E6
:10456000D1E0F0CF0E9476296C197D098E099F0950
:10457000693C71058105910528F30E9476296B013C
:104580007C01C12719F080ED97E002C080E090E047
:104590000E94AE07D7CF80E090E00E94AE07DD23F7
:1045A000B9F08091D70590E0019665E070E00E9437
:1045B000C62E8093D7050E945B0D0E94D5130E94E2
:1045C0007A0D64EF71E080E090E00E94A52909C0B7
:1045D00080E00E94DF060E94F2110E94710D0E948D
:1045E000C221DF91CF911F91FF90EF90DF90CF908C
:1045F000BF90AF909F908F900895CF92DF92EF92EF
:10460000FF9280E00E94F8070E94CF0761E089E0F6
:104610000E942F2A60E089E00E94682A61E086E01B
:104620000E942F2A61E085E00E942F2A60E08EE040
:104630000E942F2A60E08FE00E942F2A61E08FE025
:104640000E94682A60E080E10E942F2A61E080E1F8
:104650000E94682A60E088E00E942F2A61E088E0DA
:104660000E94682A61E081E10E942F2A60E081E1D6
:104670000E94682A0E949F0740E052EC61E070E0CF
:1046800086EE95E00E94CA2D0E94D5130E947A0DF5
:104690000E94BA138FEF8093AA040E94E4077894D3
:1046A0000E9476296B017C018091AA048F3F59F406
:1046B0000E9476296C197D098E099F09603D77401B
:1046C0008105910588F380ED97E00E94AE0761E0D7
:1046D0008EE00E94682A5E9A86EE95E00E94822C07
:1046E000892B29F086EE95E00E94AF2CF5CF6DEF77
:1046F00072E086EE95E00E943D2B88E893E00E94F0
:10470000620C64E173E086EE95E00E943D2B4AE086
:1047100050E064E070E086EE95E00E940D2C62E3CC
:1047200070E080E090E00E94A52986EE95E00E946E
:10473000822C04970CF186EE95E00E94AF2C823417
:104740009105D1F486EE95E00E94AF2C8E34910550
:1047500099F486EE95E00E94AF2C8434910561F4C3
:1047600086EE95E00E94AF2C819731F480E090E0D6
:104770000E94AE070E94C22140917B0550917C05AA
:1047800060917D0570917E05DB01CA010197A10949
:10479000B1090497A105B10568F44093A904433019
:1047A00029F440EA56E861E070E004C040E052ECD1
:1047B00061E070E086EE95E00E94CA2D0E945722CB
:1047C0005E9880E090E00E94AE070E94BA131092BB
:1047D000C9048091C30583FF11C080918F05882390
:1047E00051F080919605882331F080919D058823B2
:1047F00011F087E001C085E08093C90480E00E9449
:104800009C0A8091CA040E94D0090E948B0B1092CE
:104810003F0410923E0410923D04F12C8091D80583
:104820008F15B0F062E370E080E090E00E94A5296F
:1048300080ED97E00E94AE0762E370E080E090E0D8
:104840000E94A52980E090E00E94AE07F394E6CF95
:104850008091A20584FF08C0982F987181E098315B
:1048600009F080E00E94AE118FE00E94F807FF90EF
:10487000EF90DF90CF900895EF92FF920F931F93E8
:10488000CF93DF938C016EE770E086EE95E00E9497
:104890005906E801F12CF0E2EF2E8E0188818D5748
:1048A000823048F46DE770E086EE95E00E9459068C
:1048B00088818E2588832196F801608186EE95E0B7
:1048C0000E94DC2CF394F9E0FF12E7CF6EE770E072
:1048D00086EE95E00E945906CDB7DEB7E6E00C946F
:1048E000432FA9E0B0E0E7E7F4E20C942B2F90917E
:1048F000CB0491110EC09EEF99838A836B8350E0A5
:10490000559547954C832D83198618861F821E82E4
:104910002EC04091D004842F90E0B4E09595879507
:10492000BA95E1F7242F2F7030E08217930719F121
:104930008DEF89831B82FE01349650E0842F90E036
:10494000A4E095958795AA95E1F7242F2F7030E084
:104950008217930749F0DC01AF52BB4F8C918193D2
:10496000405F5F5F563051F74093D0045A83CE01C9
:1049700001960E943C248091CB0490E0019666E071
:1049800070E00E94C62E8093CB042996E2E00C943E
:10499000472FA0E0B0E0EFECF4E20C94242F6C0180
:1049A0006EE770E086EE95E00E9459068601E12CE4
:1049B000F12CC0E0D0E030E2B32EF801608183E852
:1049C000860F823078F46DE770E086EE95E00E9405
:1049D0005906F80160816B2570E086EE95E00E9433
:1049E000590604C086EE95E00E94DC2CE114F10427
:1049F00059F0F80180819E01280F311DC901C92F8E
:104A0000DD27C80FD91FDD273FEFE31AF30A89E03E
:104A1000E816F10459F028E0E216F10421F48C2F95
:104A20008095F60180870F5F1F4FC7CFCDB7DEB7E8
:104A3000E9E00C94402FA9E0B0E0E1E2F5E20C944B
:104A40002B2FE82F362F8091CB0490E0019664E263
:104A500070E00E94C62E8093CB0458E9598350E140
:104A60005A83813089F048F08230B9F08330D9F42C
:104A70008B8381EF8C833D8319C085E08B8381EF2D
:104A80008C832F5F2D8312C08B8381EF8C8384E610
:104A9000489FA00111245D8309C084E08B8381EFCE
:104AA0008C83ED8303C00E94EB1104C0CE010196FC
:104AB0000E94C9242996E2E00C94472FA2E0B0E0BE
:104AC000E4E6F5E20C94202F182F762E2A834983F2
:104AD0000E9482296B017C018091E1048090CC04CA
:104AE0009090CD04A090CE04B090CF042A8149814B
:104AF0008823C1F0D701C60188199909AA09BB0901
:104B00004C015D0191EE89169EE29906A104B10463
:104B100020F1241708F4422F202F672D812F0E94A7
:104B20001B2513C0D701C60188199909AA09BB0919
:104B30004C015D0191E3891695E79906A104B10442
:104B400060F0672D812F0E947124C092CC04D09216
:104B5000CD04E092CE04F092CF042296EDE00C94C6
:104B60003C2FA2E2B0E0E7EBF5E20C94212F8CE0C1
:104B70000E94B70981110DC06CE173E086EE95E0EB
:104B80000E946E2B5E9A80E00E949C0A0E948B0B12
:104B90005E9886EE95E00E94822C892B01F186EECC
:104BA00095E00E94AF2C9091A904992319F00E94DE
:104BB0001114EFCF40913E0450E09A012F5F3F4F18
:104BC0002F71332760913F0470E02617370709F3F0
:104BD000FA01E75BFB4F808320933E04DACF80919C
:104BE0007705843009F086C00E948229611571051D
:104BF0008105910549F06093BB047093BC048093D8
:104C0000BD049093BE040CC081E090E0A0E0B0E051
:104C10008093BB049093BC04A093BD04B093BE04E6
:104C20008091AD049091AE0481609093AE04809326
:104C3000AD0483E0809377058FE70E94950909E62C
:104C400014E00E94A809F80181938F01F4E0023773
:104C50001F07B9F72091720480916904982F922759
:104C600096FF3BC090E4922790937204982F98731C
:104C70009833F1F410E0212F30E0809169048770BF
:104C800090E0821793074CF11F5F2091A205812FBE
:104C900090E0FC01E759FB4F24FF04C080810E9493
:104CA000CD11E9CF608186EE95E00E94DC2CE3CF48
:104CB0008F7399F480916A048093B60480916B0499
:104CC0008093B40480916C048093B30480916F044A
:104CD00090E09093AC048093AB0480913D048130CC
:104CE00019F482E080933D0480913D04833011F4F7
:104CF00010923D040E9482296B017C018091AF04D7
:104D00009091B004A091B104B091B2040097A105B4
:104D1000B105C9F0A7019601281B390B4A0B5B0BA3
:104D2000DA01C901883B9B40A105B10560F00E94F2
:104D3000E6098093B5041092AF041092B00410926B
:104D4000B1041092B2048091BF049091C004A0916C
:104D5000C104B091C20446015701881A990AAA0AEF
:104D6000BB0A8AE795E00E94120886169706A806F5
:104D7000B90608F4B1C0C092BF04D092C004E0925A
:104D8000C104F092C2040E9457068091AA048830A0
:104D9000A0F08091C3059091C405A091C505B09184
:104DA000C6055CE1B695A795979587955A95D1F775
:104DB000892B8A2B8B2B09F0C4C18091AA048F5FA9
:104DC0008093AA048091BB049091BC04A091BD047F
:104DD000B091BE040097A105B105F1F0C81AD90A37
:104DE000EA0AFB0A8AE795E00E9412086C157D0525
:104DF0008E059F0508F01BC18091C30584FD04C08A
:104E000080ED97E00E94AE071092BB041092BC04A4
:104E10001092BD041092BE0490917204907C909305
:104E2000720450913E0480913F0420913D04581734
:104E300009F41AC1223009F017C1905890937204F6
:104E4000E091A205E770F0E0E658FC4F6081693020
:104E500008F0F2C0615040E04613F0C080933F0478
:104E600087E3840F90917204892B8093720440939E
:104E7000400483E080933D045D9A10918705809102
:104E8000C90481113EC18091C30582FD46C1812FB5
:104E90000E94970A8091CA040E94D009E091A2055D
:104EA000E770F0E0E658FC4F608182E794E00E94F2
:104EB000C60B8091C30582FD39C1E091CA04EF5F42
:104EC000E093CA04E83109F439C1F0E0E658FA4F3A
:104ED0008785882309F432C10E94350C813069F539
:104EE0008091A205887149F18091AD049091AE0442
:104EF000880F991F9093AE048093AD0483E0809354
:104F000077050E948B0B0E9482296093AF047093F7
:104F1000B0048093B1049093B204672B682B692B83
:104F200061F481E090E0A0E0B0E08093AF04909362
:104F3000B004A093B104B093B2048091A20584FFA1
:104F40002BC08091BB049091BC04A091BD04B09192
:104F5000BE04892B8A2B8B2BF9F08091AD049091A4
:104F6000AE048E7F0E944809182F6091AB04809197
:104F7000B6040E940714482F612F8091B50449A3FD
:104F80000E9407140091D805282F49A16091B3040D
:104F90008091B4040E945E255D988091C7048130A1
:104FA000C1F018F08230B1F1D9C08EE00E949B2A86
:104FB000892B09F0D3C081E08093C7040E94762931
:104FC0006093C3047093C4048093C5049093C60493
:104FD000C5C08EE00E949B2A892B31F50E9476295C
:104FE000C090C304D090C404E090C504F090C604FF
:104FF0006C197D098E099F09693E734081059105F1
:1050000008F4ACC082E08093C70480ED97E00E9472
:10501000AE07A4C08EE00E949B2A892B09F49EC093
:1050200080E090E00E94AE071092C70497C080E035
:1050300090E00E94AE07F0CE68E00DCF851709F42E
:105040000DCF4F5F242F30E090E0F901EE58FB4F79
:10505000DC01A75BBB4F7C917083F901E05CFB4FE7
:10506000708301968F71F8CE2430B1F42091400402
:1050700081E494E0A3E7B4E0FC013E2F381B321733
:1050800018F431913D93F9CF87E3820F9091720428
:10509000892B80937204EDCE8091C704823051F445
:1050A0009160909372045E9A8E010F5F1F4FF12CF6
:1050B000B80110C05E9880913D04811103C081E069
:1050C00080933D0480913D04833071F784E08093A8
:1050D0003D04EACF8F2D69A37AA30E943016F80110
:1050E000819391938F01F39469A17AA1F0E1FF126A
:1050F000F1CF8091A20543E754E087700E949708A2
:10510000BBCE112309F4BFCE9091C80421E0290F32
:105110002093C8049813B7CE1DC08FE00E949B2A2D
:10512000892B09F0B4CE5E9A17E0B1CE8FE00E94D1
:105130009B2A892B09F0C1CE5E98BFCE1092CA047B
:10514000CBCE8091AA04883009F45E9A89E08093DE
:10515000AA04C2CE1092C804115095CEA296ECE0DB
:105160000C943D2F8230E8F4E82FF0E0EE0FFF1FA3
:10517000E752FA4F71836083813041F0809169007A
:105180008C7F842B80936900E89A08958091690050
:10519000440F551F440F551F837F842B8093690054
:1051A000E99A08951F920F920FB60F9211242F9330
:1051B0003F934F935F936F937F938F939F93AF939F
:1051C000BF93EF93FF938091D9059091DA05892BD6
:1051D00029F0E091D905F091DA050995FF91EF9159
:1051E000BF91AF919F918F917F916F915F914F91FF
:1051F0003F912F910F900FBE0F901F9018951F9207
:105200000F920FB60F9211242F933F934F935F93FA
:105210006F937F938F939F93AF93BF93EF93FF937E
:105220008091DB059091DC05892B29F0E091DB056D
:10523000F091DC050995FF91EF91BF91AF919F919E
:105240008F917F916F915F914F913F912F910F902F
:105250000FBE0F901F9018951F920F920FB60F92CE
:1052600011242F933F938F939F93AF93BF9380917C
:10527000DE059091DF05A091E005B091E105309148
:10528000DD0523E0230F2D3720F40196A11DB11D6C
:1052900005C026E8230F0296A11DB11D2093DD0550
:1052A0008093DE059093DF05A093E005B093E105C0
:1052B0008091E2059091E305A091E405B091E505A8
:1052C0000196A11DB11D8093E2059093E305A09383
:1052D000E405B093E505BF91AF919F918F913F9108
:1052E0002F910F900FBE0F901F9018952FB7F89425
:1052F0006091DE057091DF058091E0059091E105F8
:105300002FBF08953FB7F8948091E2059091E3058F
:10531000A091E405B091E50526B5A89B05C02F3FF7
:1053200019F00196A11DB11D3FBF6627782F892F67
:105330009A2F620F711D811D911D42E0660F771F2C
:10534000881F991F4A95D1F70895CF92DF92EF9267
:10535000FF92CF93DF936B017C010E948229EB01C6
:10536000C114D104E104F10479F00E9482296C1B7C
:105370007D0B683E7340A0F381E0C81AD108E108B4
:10538000F108C851DC4FECCFDF91CF91FF90EF9047
:10539000DF90CF900895789484B5826084BD84B501
:1053A000816084BD85B5826085BD85B5816085BD20
:1053B000EEE6F0E0808181608083E1E8F0E0108239
:1053C000808182608083808181608083E0E8F0E07A
:1053D000808181608083E1EBF0E080818460808364
:1053E000E0EBF0E0808181608083EAE7F0E080819B
:1053F00084608083808182608083808181608083FB
:105400008081806880831092C1000895833081F08C
:1054100028F4813099F08230A1F008958630A9F007
:105420008730B9F08430D1F4809180008F7D03C043
:10543000809180008F7780938000089584B58F7766
:1054400002C084B58F7D84BD08958091B0008F77B0
:1054500003C08091B0008F7D8093B0000895CF93FA
:10546000DF9390E0FC01ED50F44F2491FC01E95FE3
:10547000F34F8491882349F190E0880F991FFC0134
:10548000E15DF34FA591B4918B5D934FFC01C59104
:10549000D4919FB7611108C0F8948C912095822314
:1054A0008C93888182230AC0623051F4F8948C91E5
:1054B000322F309583238C938881822B888304C07C
:1054C000F8948C91822B8C939FBFDF91CF9108959C
:1054D000A1E0B0E0EEE6FAE20C94292F282F30E0AC
:1054E000F901E152F44F8491F901ED50F44F149118
:1054F000F901E95FF34F04910023C9F0882321F0FB
:1055000069830E94062A6981E02FF0E0EE0FFF1FF9
:10551000EB5DF34FA591B4919FB7F8948C91611115
:1055200003C01095812301C0812B8C939FBF2196CE
:10553000E4E00C94452FCF93DF93282F30E0F9015E
:10554000E152F44F8491F901ED50F44FD491F901F7
:10555000E95FF34FC491CC2391F081110E94062A98
:10556000EC2FF0E0EE0FFF1FE55EF34FA591B49135
:105570002C912D2381E090E021F480E002C080E0B6
:1055800090E0DF91CF9108958E3008F08E508770B3
:1055900020919D0190E4299F90011124822B8093FA
:1055A0007C0080917A00806480937A0080917A00F8
:1055B00086FDFCCF809178002091790090E0922BBD
:1055C0000895A0E0B0E0E7EEFAE20C94252F6C011C
:1055D0007A01EB01E60EF71E00E010E0CE15DF05C4
:1055E00061F06991D601ED91FC910190F081E02D7F
:1055F000C6010995080F191FF1CFC801CDB7DEB755
:10560000E8E00C94412F6115710589F0DB010D90E4
:105610000020E9F7AD0141505109461B570BDC0151
:10562000ED91FC910280F381E02D0995089580E0D1
:1056300090E00895EF92FF920F931F93CF93DF9323
:105640008C01FB01C0E0D0E064917F018FEFE81A8C
:10565000F80A662361F0D801ED91FC910190F08188
:10566000E02DC8010995C80FD91FF701EDCFCE0174
:10567000CDB7DEB7E6E00C94432F0E94032B0895CC
:10568000DC01ED91FC910190F081E02D09950895E8
:105690000F931F93CF93DF93EC016DE00E94402B9B
:1056A0008C016AE0CE010E94402B800F911FDF9198
:1056B000CF911F910F9108950F931F93CF93DF9375
:1056C000EC010E941A2B8C01CE010E94482B800F06
:1056D000911FDF91CF911F910F9108950F931F9309
:1056E000CF93DF93EC010E94032B8C01CE010E942B
:1056F000482B800F911FDF91CF911F910F9108953B
:105700000F931F93CF93DF93EC010E94402B8C01EA
:10571000CE010E94482B800F911FDF91CF911F91E6
:105720000F910895A1E2B0E0E8E9FBE20C94212F8B
:105730007C01C42EE52FCB01D22E19A221E02D151C
:1057400010F02AE0D22E8E010F5D1F4F8D2C912C70
:10575000A12CB12C6C2D7E2FA50194010E94DA2E74
:105760008C2DD29E80191124015011098A3010F419
:10577000805D01C0895CF8018083211531054105F8
:10578000510521F0C22EE32FCA01E4CFB801C701B1
:105790000E94032BA196ECE00C943D2FA0E0B0E01A
:1057A000E4EDFBE20C94252FEC016A017B0121154D
:1057B000310541F4E881F9810190F081E02D642FF9
:1057C00009951DC02A303105A9F477FF12C06DE29A
:1057D0000E94402B8C0144275527BA014C195D09C2
:1057E0006E097F092AE0CE010E94922B800F911F43
:1057F00006C02AE0B701A601CE010E94922BCDB7C8
:10580000DEB7E8E00C94412F9A01AB01662757FD03
:105810006095762F0E94CE2B08950F931F93CF9300
:10582000DF93EC019A01AB01662757FD6095762F57
:105830000E94CE2B8C01CE010E94482B800F911F1D
:10584000DF91CF911F910F9108952115310549F4F2
:10585000DC01ED91FC910190F081E02D642F099520
:1058600008950E94922B08959A01462F50E060E01F
:1058700070E00E94252C08959A01AB0160E070E071
:105880000E94252C08950F931F93CF93DF93EC0173
:105890000E94252C8C01CE010E94482B800F911F65
:1058A000DF91CF911F910F9108950F931F93CF9385
:1058B000DF93EC019A01AB0160E070E00E94252CBF
:1058C0008C01CE010E94482B800F911FDF91CF9158
:1058D0001F910F9108950F931F93CF93DF93EC01C6
:1058E0009A01462F50E060E070E00E94252C8C0168
:1058F000CE010E94482B800F911FDF91CF911F9105
:105900000F910895FC0124853585F901E05CFF4F76
:1059100080819181F901EE5BFF4F20813181821BF3
:10592000930B8F7399270895FC0184859585FC015D
:10593000E05CFF4F40815181FC01EE5BFF4F208115
:1059400031814217530741F00190F081E02DE80FBB
:10595000F91F808190E008958FEF9FEF0895FC017B
:1059600084859585FC01E05CFF4F40815181FC01FD
:10597000EE5BFF4F208131814217530779F0A08100
:10598000B181A80FB91F8C91208131812F5F3F4FCA
:105990002F7333273183208390E008958FEF9FEF9B
:1059A0000895FC0181A1882329F0A489B5898C91EF
:1059B00086FFFBCF11A20895CF93DF93FC012685CC
:1059C0003785D901A05CBF4F8D919C9111970196AD
:1059D0008F739927E901CE5BDF4F48815981841786
:1059E0009507D9F30D90BC91A02DA20FB31F6C9316
:1059F000A685B785A05CBF4F11969C938E93A68910
:105A0000B7892C9181E090E0078C02C0880F991F24
:105A10000A94E2F7282B2C9381E081A30488F5896E
:105A2000E02D80818064808381E090E0DF91CF91E0
:105A3000089508951F920F920FB60F9211242F937D
:105A40003F934F938F939F93EF93FF938091C00069
:105A500082FD1CC04091C60080918C0690918D06FD
:105A600001968F73992720918E0630918F068217A9
:105A7000930771F0E0918C06F0918D06E45BF94F8D
:105A8000408390938D0680938C0602C08091C6005F
:105A9000FF91EF919F918F914F913F912F910F9097
:105AA0000FBE0F901F90189586EE95E00E94822CF5
:105AB000892B11F00E94192D08951F920F920FB695
:105AC0000F9211242F933F938F939F93EF93FF9304
:105AD000209148063091490680914A0690914B06E4
:105AE0002817390731F48091C1008F7D8093C10060
:105AF00014C0E0914A06F0914B06E85FF94F20810F
:105B000080914A0690914B0601968F739927909346
:105B10004B0680934A062093C600FF91EF919F9118
:105B20008F913F912F910F900FBE0F901F9018955E
:105B3000A0E0B0E0EEE9FDE20C94212FFC0113821D
:105B4000128288EE93E0A0E0B0E084839583A68380
:105B5000B7838CEB93E09183808375876487578745
:105B60004687318B208B138B028BF58AE48AD78A88
:105B7000C68AB18EA08E938E828E8F85848F8889FF
:105B8000858F8989868F8A89878F8B8980A3ECE0AE
:105B90000C943D2FCF92DF92EF92FF92CF93DF9341
:105BA000EC016A017B01411581EE58076105710521
:105BB000F9F0EC89FD8981E090E008A002C0880F2F
:105BC000991F0A94E2F7808360E079E08DE390E02A
:105BD000A70196010E94DA2E21503109410951098D
:105BE0005695479537952795211580E1380798F008
:105BF000EC89FD89108260E874E88EE190E0A701ED
:105C000096010E94DA2E2150310941095109569519
:105C1000479537952795E889F9893083EA89FB8983
:105C2000208319A2EE89FF89408181E090E09C01E8
:105C30000C8C02C0220F331F0A94E2F7422B4083E0
:105C4000EE89FF8940819C010D8C02C0220F331F19
:105C50000A94E2F7422B4083EE89FF8940819C0140
:105C60000E8C02C0220F331F0A94E2F7422B4083AE
:105C7000EE89FF8920810F8C02C0880F991F0A943A
:105C8000E2F7809582238083DF91CF91FF90EF90A0
:105C9000DF90CF9008958F929F92AF92BF92CF9254
:105CA000DF92EF92FF920F931F9381E08F9385E035
:105CB0008F9387E08F9383E08F9384E08F93E6EC5C
:105CC0008E2E912CF2ECAF2EB12CA1ECCA2ED12C41
:105CD000B0ECEB2EF12C04EC10E025EC30E048E0C9
:105CE00056E06CE476E086EE95E00E94982D0F90E9
:105CF0000F900F900F900F901F910F91FF90EF90CA
:105D0000DF90CF90BF90AF909F908F9008950E94AA
:105D1000CB290E94FD22C4E5DDE20E94B125209737
:105D2000E1F30E94542DF9CFA29FB001B39FC001AF
:105D3000A39F700D811D1124911DB29F700D811DB7
:105D40001124911D08950E94942EA59F900DB49F3B
:105D5000900DA49F800D911D11240895B7FF0C9400
:105D6000A32E0E94A32E821B930B0895DB018F9319
:105D70009F930E94A32EBF91AF91A29F800D911D72
:105D8000A39F900DB29F900D1124089597FB072EAD
:105D900016F4009407D077FD09D00E94582F07FC15
:105DA00005D03EF4909581959F4F0895709561952B
:105DB0007F4F0895A1E21A2EAA1BBB1BFD010DC047
:105DC000AA1FBB1FEE1FFF1FA217B307E407F507AB
:105DD00020F0A21BB30BE40BF50B661F771F881F87
:105DE000991F1A9469F760957095809590959B011D
:105DF000AC01BD01CF010895052E97FB1EF4009460
:105E00000E94132F57FD07D00E94DA2E07FC03D003
:105E10004EF40C94132F50954095309521953F4F9B
:105E20004F4F5F4F089590958095709561957F4F86
:105E30008F4F9F4F08952F923F924F925F926F9294
:105E40007F928F929F92AF92BF92CF92DF92EF920A
:105E5000FF920F931F93CF93DF93CDB7DEB7CA1B8B
:105E6000DB0B0FB6F894DEBF0FBECDBF09942A88B6
:105E7000398848885F846E847D848C849B84AA845E
:105E8000B984C884DF80EE80FD800C811B81AA81EB
:105E9000B981CE0FD11D0FB6F894DEBF0FBECDBFB6
:105EA000ED010895EE0FFF1F0590F491E02D099488
:105EB000AA1BBB1B51E107C0AA1FBB1FA617B70730
:105EC00010F0A61BB70B881F991F5A95A9F780954C
:105ED0009095BC01CD0108958F929F92AF92BF9291
:105EE000CF92DF92EF92FF92CF93DF93EC01688124
:105EF00079818A819B81611571058105910521F464
:105F000064E279ED8BE597E02DE133EF41E050E07D
:105F10000E94FC2E49015A019B01AC01A7EAB1E4A1
:105F20000E94A32E6B017C01ACEEB4EFA50194019D
:105F30000E94B12EC60ED71EE81EF91EF7FE06C03F
:105F400081E0C81AD108E10880E8F80AC882D9823D
:105F5000EA82FB82C701B6019F77DF91CF91FF9064
:105F6000EF90DF90CF90BF90AF909F908F9008956B
:105F70000E946C2F089586E091E00E946C2F089596
:105F800060930601709307018093080190930901C3
:105F900008952F923F925F926F927F928F929F927D
:105FA000AF92BF92CF92DF92EF92FF920F931F9327
:105FB000CF93DF938B01EA016115710521F0DB01BD
:105FC0008C9311969C93209739F09E0122503109B1
:105FD0002332310508F0D8C07C016701BFEFCB1A2E
:105FE000DB0A5601F7016080862D90E00E94FB30AD
:105FF000892B11F07601F1CFFDE26F120AC0570133
:1060000082E0A80EB11CD70111966C90772473948E
:106010000BC0BBE26B1207C05701E2E0AE0EB11C31
:10602000D70111966C90712CCE018F7E892B89F44B
:10603000B0E36B1237C0F50180818F7D8835D1F4D4
:106040006180F2E0AF0EB11C872D8260782EC0E136
:10605000D0E0CA30D10551F1C031D10521F0C830AE
:10606000D10599F409C0CC24CA94DC2CEC2CAFE007
:10607000FA2E22C0209769F7C8E0D0E0CC24CA9459
:10608000DC2CEC2CFFE1FF2E17C06FEF7FEFCB0174
:106090009E01442737FD4095542F0E94DA2E690156
:1060A0007A010AC02097A9F6CAE0D0E0E9E9CE2E2D
:1060B000DC2CEC2CE9E1FE2EF50160E020E030E084
:1060C000A9014E01AA2497FCA094BA2C1F0170EDDF
:1060D000572E560CA9E0A51570F48FEB860D8A316A
:1060E00018F499EC592E06C08FE9860D8A3148F5CF
:1060F00089EA582E560C852D90E08C179D070CF5DB
:106100006F3FD9F0C216D306E406F50698F0C50134
:10611000B4010E94B62E9B01AC01852D90E0A0E059
:10612000B0E0280F391F4A1F5B1F281739074A079D
:106130005B0710F46FEF01C061E03196D1016C9004
:10614000C5CF0115110551F0662311F0319703C039
:1061500071FE04C03297D801ED93FC9370FE07C026
:1061600050954095309521953F4F4F4F5F4F67FFBA
:1061700010C082E290E090939106809390066FEFBA
:106180007FEF8FEF9FEF07C060E070E080E090E06E
:1061900002C0B901CA01DF91CF911F910F91FF9009
:1061A000EF90DF90CF90BF90AF909F908F907F90B7
:1061B0006F905F903F902F900895FC01882799275A
:1061C000E89421912032E9F3293010F02E30C8F301
:1061D0002B3241F02D3239F4689404C00E942F31E3
:1061E000820F911D219120532A30C0F31EF4909507
:1061F00081959F4F0895911150C0803219F08950B8
:106200008550D0F7089548EC53E00E940831089576
:10621000FA01A191B081009719F41097E1F0CD0136
:10622000DC01CD010D90002011F4C00113C0FB0171
:106230002191222319F02015D9F7F3CFFB012191E9
:10624000201519F41E92119606C02223C1F70D9055
:106250000020A1F7D001FA01A193B08308957AE05C
:10626000979F902D879F802D910D11240895F99966
:10627000FECF92BD81BDF89A992780B50895262F4B
:10628000F999FECF1FBA92BD81BD20BD0FB6F8941B
:10629000FA9AF99A0FBE01960895992788270895CA
:0462A000F894FFCFA0
:1062A40000009206200001000000FF00020002002E
:1062B40002000200020002000200020002000200CA
:1062C4000200020002000200020002802500000514
:1062D400400AA1204EA50020244EA52C2330C01234
:1062E40000001A400AA1204EA5001B1E27522C2391
:1062F400308025000005400AA1204EA50020244E30
:10630400A52C2330004B000006400AD0009D490014
:106314007B289D492C233000E1000005400A4501FB
:10632400D7DC03B81E0EBF00232E48E801008A40C4
:106334000A6001555502AD1E20000023C8015458BF
:106344002074696D656F75742100596573004E6F13
:10635400002C00386368004E2F41002C205B005D48
:106364002028002900486F70206368616E6E656C98
:10637400200020402000456E746572696E672061BC
:1063840064617074697665206368616E6E656C2003
:1063940073656C656374696F6E2C207069636B69D7
:1063A4006E673A007363616E6E6572206D6F64652B
:1063B400004E4F5420454E41424C45440053656EB7
:1063C40064696E672073657474696E677320746F93
:1063D4002052580A00526573657474696E6720739D
:1063E400657474696E6773206F6E2052580A004199
:1063F400626F727465642065646974730A00696EFF
:1064040076616C69642073656C656374696F6E0092
:106414000D0A496E76616C696420696E707574202A
:106424002D20646973636172646564210700536598
:106434007474696E677320736176656420746F2069
:10644400454550524F4D0A00526576657274656435
:106454002073657474696E67732066726F6D20456E
:106464004550524F4D0A004C6F616465642066616B
:1064740063746F72792064656661756C74730A0065
:106484004B657920616E64206368616E6E656C7320
:106494002072616E646F6D697A65640A004F70657D
:1064A4006E4C52536E672054582073746172746931
:1064B4006E672000206F6E20485720006D6F647552
:1064C4006C65206C6F636B65643F00342B3400385B
:1064D40000382B340031320031322B340031360095
:1064E40050504D0052535349005344410053434CC0
:1064F40000525844005458440041494E004C42450F
:1065040045500053504B54524D0053425553005381
:10651400554D44004C4C494E440000070B0C1011DF
:106524001500B7012B032F033103350338033D0353
:10653400B7014003440349034D0351035503590371
:106544005D0363036A036F0374038D028D028D027E
:106554008D02160A1322312900000000DC2CE12AE6
:08656400822CAF2C942CD12CE9
:107E00000F92CDB7DEB7112484B714BE81FFF1D035
:107E100082E08093C00088E18093C10086E0809377
:107E2000C20080E18093C4008EE0CDD088249924E4
:107E3000CC24C394F5E0DF2EE1E1EE2E73E0F72EC3
:107E4000B6D0082F813479F4B2D08983C2D0898129
:107E5000823811F481E005C0813811F485E001C059
:107E600083E09ED09AC0823411F484E103C085344B
:107E700019F485E0B6D091C0853561F498D0082F0B
:107E800010E095D090E0982E8824802A912A880CC2
:107E9000991C82C0863521F484E0A3D080E0E1CF34
:107EA000843609F04CC083D082D0A82E80D0B82E62
:107EB00000E011E07CD0F80181938F01AE16D1F77C
:107EC00088D0FB2DF53489F4E0E0F1E00BC0F9999E
:107ED000FECF92BC81BC0894811C911C819180BD15
:107EE000FA9AF99AEA1598F358C08B2D863409F05E
:107EF00054C0F401F7BEE89507B600FCFDCFF401CD
:107F0000A0E0B1E02C9130E011968C91119790E0B7
:107F1000982F8827822B932B12960C01C7BEE895C9
:107F20001124329681E0A038B80761F7F401D7BE7A
:107F3000E89507B600FCFDCFE7BEE8952EC0843774
:107F4000F1F435D034D0182F32D0B82E42D0FB2DDA
:107F5000F63421F4F40105914F010CC0FB2DF534EA
:107F600049F4F999FECF92BC81BC0894811C911C04
:107F7000F89A00B5802F14D0115049F70EC08537FC
:107F800039F427D08EE10CD085E90AD08FE069CF93
:107F9000813511F488E017D01CD080E101D050CF9A
:107FA0009091C00095FFFCCF8093C600089580910A
:107FB000C00087FFFCCF8091C00084FD01C0A89560
:107FC0008091C6000895E0E6F0E098E19083808318
:107FD0000895EDDF803219F088E0F5DFFFCF84E10E
:107FE000DFCF1F93182FE3DF1150E9F7F2DF1F9166
:0E7FF0000895282E80E0E7DFEE27FF27099492
:027FFE0001057B
:0400000300007E007B
:00000001FF
